:100000000C9407040C942F040C942F040C942F04CC
:100010000C942F040C942F040C94E8360C942F04A9
:100020000C942F040C942F040C942F040C942F0484
:100030000C942F040C942F040C94A0380C94513978
:100040000C942F040C942F040C942F040C942F0464
:100050000C9479360C942F040C942F040C942F04D8
:100060000C949E360C9409380C9433370C940D374D
:100070000C942F040C942F360C942F040C942F0402
:100080000C942F040C942F040C94C3360C94543607
:100090000C94A5370C947F370C9459370C942F048B
:1000A00007634236B79BD8A71A39685618AEBAAB61
:1000B000558C1D3CB7CC5763BD6DEDFD753EF617F5
:1000C0007231BF000000803F08000000BE9224494A
:1000D000123EABAAAA2ABECDCCCC4C3E000000807A
:1000E000BEABAAAAAA3E00000000BF000000803FED
:1000F0000000000000084178D3BB4387D1133D19AD
:100100000E3CC3BD4282AD2B3E68EC8276BED98FD9
:10011000E1A93E4C80EFFFBE01C4FF7F3F0000001D
:100120000000010008191304E81A0010191302E86E
:100130004C0011191301E8820010191301E8B400F2
:1001400011191301E8EA0010191302E81C01101933
:100150001302E84E0111191301E8000303070F3FD2
:10016000FFFF07070707070707070707070707072F
:100170000707070707E01FF83FFC7C3E700FF00FF2
:10018000E007E00700070007000F001E003C00F832
:1001900003F007C01F003C00380070006000E00062
:1001A000FFFFFFFFFFFF07F007FE07FF8783C38006
:1001B000F38039C01CE00E0007000F007F003F00F5
:1001C0001FE00078001E00070003F001F800FE00A9
:1001D000770073E0F8FFF83FF807F00000380038C8
:1001E000007800F800F801F803B8033807380E3833
:1001F0001C381838383870386038E038FFFFFFFF97
:10020000FFFF0038003800380038003800381FFF82
:100210000FFF8FFFC700038001C000E000700039AE
:10022000F03FFE1FFF8F83E700F0003C000E000749
:1002300000038001C000FC00EF0073C0F0FFF83F36
:10024000F807E00003E00FF81FFC3C1E380E700EAC
:1002500070006000E000E3E0EFF8FFFCFC3EF00E11
:10026000F00FE007E007E0076007700F700E3C3EFC
:100270003FFC1FF807E0FFFFFFFFFFFF0006000E37
:10028000001C001800380070006000E000C001C0D1
:100290000180038003800700070007000E000E00A6
:1002A0000E000C001C001C0007F00FFE0FFF8783E0
:1002B000C780F38039C01CE00E780F1E0F07FF01C6
:1002C000FF03FFE3E0F9C01DC00FE003F001F800F9
:1002D000FC00F70073E0F8FFF83FF807F000005A61
:1002E000012201310038003800000000003E5B4F61
:1002F0005B3E3E6B4F6B3E1C3E7C3E1C183C7E3C86
:10030000181C577D571C1C5E7F5E1C00183C180093
:10031000FFE7C3E7FF0018241800FFE7DBE7FF3023
:10032000483A060E2629792926407F050507407F91
:1003300005253F5A3CE73C5A7F3E1C1C08081C1C04
:100340003E7F14227F22145F5F005F5F06097F01FA
:100350007F006689956A606060606094A2FFA294E5
:1003600008047E040810207E201008082A1C0808B3
:100370001C2A08081E101010100C1E0C1E0C303801
:100380003E3830060E3E0E06000000000000005F02
:1003900000000007000700147F147F14242A7F2A1E
:1003A00012231308646236495620500008070300E0
:1003B000001C2241000041221C002A1C7F1C2A082C
:1003C000083E08080080703000080808080800008F
:1003D00060600020100804023E5149453E00427F03
:1003E000400072494949462141494D331814127F52
:1003F0001027454545393C4A4949314121110907F2
:100400003649494936464949291E00001400000072
:100410004034000000081422411414141414004144
:1004200022140802015909063E415D594E7C121101
:10043000127C7F494949363E414141227F41414139
:100440003E7F494949417F090909013E41415173B4
:100450007F0808087F00417F41002040413F017F25
:10046000081422417F404040407F021C027F7F04ED
:1004700008107F3E4141413E7F090909063E415136
:10048000215E7F09192946264949493203017F0126
:10049000033F4040403F1F2040201F3F4038403F27
:1004A000631408146303047804036159494D43003D
:1004B0007F4141410204081020004141417F040274
:1004C000010204404040404000030708002054540B
:1004D00078407F28444438384444442838444428E9
:1004E0007F385454541800087E090218A4A49C783C
:1004F0007F0804047800447D40002040403D007F98
:100500001028440000417F40007C047804787C0877
:100510000404783844444438FC182424181824244B
:1005200018FC7C08040408485454542404043F4430
:10053000243C4040207C1C2040201C3C4030403C5F
:1005400044281028444C9090907C4464544C4400BF
:100550000836410000007700000041360800020123
:100560000204023C2623263C1EA1A161123A40400F
:10057000207A38545455592155557941225454788C
:1005800042215554784020545579400C1E52721225
:1005900039555555593954545459395554545800AE
:1005A00000457C410002457D420001457C407D12B2
:1005B00011127DF0282528F07C5455450020545414
:1005C0007C547C0A097F4932494949323A444444BF
:1005D0003A324A4848303A4141217A3A42402078FA
:1005E000009DA0A07D3D4242423D3D4040403D3CFB
:1005F00024FF2424487E4943662B2FFC2F2BFF0920
:1006000029F620C0887E0903205454794100004413
:100610007D413048484A32384040227A007A0A0AFE
:10062000727D0D19317D2629292F28262929292671
:1006300030484D4020380808080808080808382FB6
:1006400010C8ACBA2F102834FA00007B0000081440
:100650002A142222142A14085500550055AA55AA16
:1006600055AAFF55FF55FF000000FF00101010FFB6
:1006700000141414FF001010FF00FF1010F010F011
:10068000141414FC001414F700FF0000FF00FF1402
:1006900014F404FC141417101F10101F101F14144E
:1006A000141F00101010F0000000001F1010101098
:1006B0001F10101010F010000000FF10101010108C
:1006C00010101010FF10000000FF140000FF00FFCA
:1006D00000001F10170000FC04F414141710171466
:1006E00014F404F40000FF00F71414141414141488
:1006F000F700F7141414171410101F101F141414FB
:10070000F4141010F010F000001F101F0000001F64
:1007100014000000FC140000F010F01010FF10FF97
:10072000141414FF141010101F00000000F010FF2C
:10073000FFFFFFFFF0F0F0F0F0FFFFFF0000000010
:1007400000FFFF0F0F0F0F0F3844443844FC4A4A94
:100750004A347E02020606027E027E026355494149
:10076000633844443C04407E201E2006027E020280
:1007700099A5E7A5991C2A492A1C4C7201724C3094
:100780004A4D4D303048784830BC625A463D3E496B
:100790004949007E0101017E2A2A2A2A2A44445F0F
:1007A000444440514A444040444A51400000FF0103
:1007B00003E080FF000008086B6B08361236243611
:1007C000060F090F06000018180000001010003076
:1007D00040FF0101001F01011E00191D1712003CFE
:1007E0003C3C3C00000000000901809611800A3A60
:1007F00081550A3601082A04000000F02B0400008D
:10080000014021800A13800A29800A00113A11242C
:100810001FBECFEFCDBFDFE3DEBF18E2A0E0B8E23E
:10082000E1EFF0EB02C005900D92A637B107D9F7C2
:100830002EE2A6E7B8E201C01D92AB30B207E1F7A5
:1008400014E0C7E0D4E004C02197FE010E9459558E
:10085000C630D107C9F70E94AB3B0C94C1560C942B
:10086000000090E0FC01EA57F141E081EF3F39F1EF
:10087000865E9041DC012C91822F880F880F880FB3
:100880008E0F8033E0F490E0880F991FDC01A75BA6
:10089000B44D6D937C938751954DDC011D921C9254
:1008A000B0E22B9FC00111249C5F4096E80FF92F06
:1008B000F11D8081887F808380818160808308959D
:1008C000CF93C82F8091B82D9091B92DDC01ED9177
:1008D000FC910688F789E02D6091B72D09958091EC
:1008E000B82D9091B92DDC01ED91FC910190F08132
:1008F000E02D6C2F09958091B82D9091B92DDC01D8
:10090000ED91FC91028CF38DE02D0995882331F057
:1009100082E88093BA2D80E0CF9108958091B82D20
:100920009091B92DDC01ED91FC91048CF58DE02DB9
:1009300021E041E050E06091B72D0995813041F709
:100940001092BA2D8091B82D9091B92DDC01ED91C6
:10095000FC910284F385E02D0995DECFCF93DF93E0
:10096000D82FC62F8091B82D9091B92DDC01ED9133
:10097000FC910688F789E02D6091B72D099580914B
:10098000B82D9091B92DDC01ED91FC910190F08191
:10099000E02D6D2F09958091B82D9091B92DDC0136
:1009A000ED91FC910190F081E02D6C2F09958091E3
:1009B000B82D9091B92DDC01ED91FC91028CF38D55
:1009C000E02D0995882339F082E88093BA2D80E0E4
:1009D000DF91CF9108951092BA2D81E0F9CFCF9396
:1009E000DF93D82FC62F89E00E9460049091BA2D22
:1009F000911112C061E070E001C0660FDA95EAF76C
:100A0000CC2371F0682B861771F089E00E94AE0448
:100A100081E09091BA2D911180E0DF91CF910895FE
:100A200060956823F0CF81E0F8CFCF93DF93D82F84
:100A3000C62F80E00E9460049091BA2D911110C0E1
:100A400061E070E001C0660FDA95EAF7C23061F448
:100A5000682B80E00E94AE0481E09091BA2D911144
:100A600080E0DF91CF91089560956823F2CFFC017B
:100A700054894589252F30E0842F90E0821B930B09
:100A8000541710F0CF96089501970895FC019289AC
:100A90008389981761F0A389AE0FBF2FB11D5996B6
:100AA0008C9193899F5F9F73938B90E008958FEF54
:100AB0009FEF0895FC0192898389981731F083890B
:100AC000E80FF11D818D90E008958FEF9FEF08955D
:100AD000FC0192892389892F90E0805C9F4F821BC3
:100AE00091098F7399270895CF93DF93EC01E881E3
:100AF000F9810680F781E02D0995EC85FD858681D9
:100B00008F738683EC85FD8585818F7585838B89C1
:100B10008A8B198ADF91CF910895CF93DF93FC01DF
:100B200094898589C485D585981306C08D818F7D6C
:100B30008D83DF91CF910895A589AE0FBF2FB11D91
:100B4000A75ABF4F2C91858990E001968F73992702
:100B5000858B80E48C83A485B58512962C9394892B
:100B600085899813E6CFA485B58515968C91159740
:100B70008F7D15968C9387898823D9F2808D8093F9
:100B80001301178AD6CFDC011C96ED91FC910FB6AC
:100B900007FE03C0258125FD04C0248125FD0C949A
:100BA0008D050895EF92FF920F931F93CF93DF93DC
:100BB000EC0181E0898B9C898D8998131CC0AC85E0
:100BC000BD8514968C91149785FF15C012966C9371
:100BD000AC85BD8580E414968C93EC85FD8585817C
:100BE0008F7D858381E090E0DF91CF911F910F9100
:100BF000FF90EF9008958091110180FF08C08091CF
:100C00001301888F8E898093130181E08F8BF62EDC
:100C10000C8910E00F5F1F4F0F731127E02E8D8995
:100C20008E1104C0CE010E94C305F9CFEC89EC0FF0
:100C3000FD2FF11DE75AFF4FF0820C8BEC85FD85EF
:100C400085818062CECFCF93DF93FC01218922235F
:100C5000C9F0EC018091110180FF08C0809113015F
:100C6000808F86898093130181E0878BEC85FD85D9
:100C7000858185FD03C0848186FD04C0CE010E946C
:100C8000C305F4CFDF91CF910895AF92BF92CF9279
:100C9000DF92EF92FF920F931F93CF93DF936C013C
:100CA0007B018B01040F151FEB015E01AE18BF081D
:100CB000C017D10759F06991D601ED91FC910190CF
:100CC000F081E02DC6010995892B79F7C501DF91E7
:100CD000CF911F910F91FF90EF90DF90CF90BF9039
:100CE000AF900895EF92FF920F931F93CF93DF93EE
:100CF000C82FD0E0A09695E0CC0FDD1F9A95E1F7C4
:100D0000E984F82EFF0CFF0CFF0C01E010E08E2DA3
:100D10008023A9F02F2D210F30E0220F331FF9017E
:100D2000E75BF44D80819181892B49F00190F0813E
:100D3000E02D2751354DD9018D919C9109951F5F6B
:100D4000000F183021F7E986DF91CF911F910F91A5
:100D5000FF90EF900895FC01A485B58511968C91C4
:100D6000119781FD1BC06C9182898F5F8F7393896E
:100D7000981739F0A289AE0FBF2FB11D59966C9309
:100D8000828BE756FF4F80819181009741F0DC0113
:100D9000ED91FC910190F081E02D09948C910895E2
:100DA00081E00895CF93DF9390E0FC01E050F141A2
:100DB00020812F3F89F06330710570F4FC01E65EFD
:100DC000F041A08130E2A39FD0011124BC5F6130CB
:100DD000710529F411962C93DF91CF9108958A57CC
:100DE0009141EC01E881EF3F89F0CD014096E80F99
:100DF000F92FF11D9FB7F89412962C9380816230E1
:100E0000710539F4886080839FBFE6CFF0E0E0E0B1
:100E1000F1CF877FF8CF8B3210F40C94D20608956F
:100E2000282F30E0F901EA5DF141E081EE2309F17C
:100E3000E13021F0F0F0E63098F008954091010A99
:100E40002A573141F90120812C5F81E090E001C0F7
:100E5000880F2A95EAF7809584238093010A0895E4
:100E600080E1E89FF0011124E05AF54F81818F7EE7
:100E700081830895FF920F931F93CF93DF93082FE1
:100E800010E0F801E050F141F0809FEFF916A1F079
:100E9000EB018B3210F40E941007F801E65EF0417E
:100EA000E08180E2E89FF0011124FC5F80818F21C6
:100EB00079F0209739F4F682DF91CF911F910F914D
:100EC000FF900895229711F4F782F6CFF582F4CFC0
:100ED000D801AA57B1418C91309771F08F3F61F0E2
:100EE0007096E80FF11D9FB7F8948081CD2B39F4EF
:100EF000877F80839FBFE0CFF0E0E0E0F4CF8860A1
:100F0000F8CF8B3210F40C943A070895CF92DF9209
:100F1000EF92FF920F931F93CF93DF93EC016A013F
:100F20007B01022F8989882339F0E881F9810288C1
:100F3000F389E02DCE01099598898091E205892BEE
:100F40008093E2051FB7F89460E070E281EA97E0D1
:100F5000A70196010E94C75069017A018FEFC81A54
:100F6000D80AE80AF80AF694E794D794C794EC856F
:100F7000FD8586818D7F8683EC85FD8586818683D0
:100F8000198AA09123110A2E000CBB0BA701960110
:100F90000E948E5020E034E040E050E00E94645017
:100FA000EC85FD85C20ED31EE41EF51EC086D186DB
:100FB000EC85FD850783EC85FD858681806C8683C5
:100FC000EC85FD858581806885838E8562E070E093
:100FD0000E940B078F8561E070E00E9481078F857A
:100FE00061E070E00E940B071FBFDF91CF911F915E
:100FF0000F91FF90EF90DF90CF9008950F931F9384
:10100000CF93082F10E0F801E050F141C081CF3FAD
:10101000B9F08B3210F40E941007F801E65EF0413F
:10102000E08180E2E89FF0011124FC5F8085C82305
:1010300081E090E009F480E0CF911F910F91089535
:1010400080E090E0F9CFE82FF0E0E25EF1418E30F1
:10105000B8F480818F30B0F48093060681E08093ED
:10106000080680910B0680FFFCCF2FB7F894909173
:101070001006809111062FBF892798278927089588
:101080003E97E7CF8FEF90E00895CF93DF938FB730
:10109000F8942091492A30914A2A40914B2A509144
:1010A0004C2AE091BA0A9091B60A90FF06C02F5FD1
:1010B0003F4F4F4F5F4FE091BA0A8FBFA091532A25
:1010C000B091542AC091512AD091522A0E94835043
:1010D000EC9F9001ED9F300D1124620F731F811D55
:1010E000911DDF91CF9108958F929F92AF92BF9201
:1010F000CF92DF92EF92FF924B015C010E94450874
:101100006B017C01A8EEB3E0A50194010E9483501D
:10111000C60ED71EE81EF91EC616D706E806F90643
:1011200018F40E944508F8CF0E9445086C157D050B
:101130008E059F05C8F3FF90EF90DF90CF90BF9092
:10114000AF909F908F9008952FB7F8946091452AA3
:101150007091462A8091472A9091482A2FBF08957E
:101160000F931F93CF93DF938C01EB0180915C2849
:1011700090915D28A0915E28B0915F28892B8A2BE1
:101180008B2B51F40E94A40860935C2870935D2817
:1011900080935E2890935F280130110539F0CF3F8E
:1011A000DC07A1F481E08093612806C0CF3FDC0713
:1011B00041F481E080936028DF91CF911F910F91DE
:1011C0000895C0936528D0936628F6CFC09363280E
:1011D000D0936428F1CF8F929F92AF92BF92EF92FB
:1011E000FF921F93CF93DF93182FEB017A0189E0D1
:1011F0000E9460049091BA2D911137C021E030E037
:1012000001C0220F1A95EAF7822311E009F410E0D9
:101210000E94A40811114FC088809980AA80BB80C9
:1012200081149104A104B10411F5688379838A8340
:101230009B838F8198850297029760F4112351F068
:10124000F701878190850297029720F48185928526
:1012500087839087812FDF91CF911F91FF90EF902F
:10126000BF90AF909F908F9008951FEFD1CF1D81B9
:10127000111167C0681979098A099B096D3271409B
:101280008105910590F081E08D838F819885823072
:10129000910598F18430910508F040C02D812223FA
:1012A00009F448C081E08E8339C08C818111C1CF9F
:1012B00081E08C83BECF1C811123B9F02D812111D7
:1012C00013C088809980AA80BB80681979098A092F
:1012D0009B0989889A88092C000CAA08BB088616E5
:1012E0009706A806B90688F210E01C821D821E82AD
:1012F000188219821A821B829CCF89879A872D8136
:10130000222399F0019771F083E090E08F83988712
:101310000E94A4086B877C878D879E871111E5CF7B
:1013200011E087CF82E090E0F1CFE1E08E278F835C
:101330009887F4CF29853A8589879A872F833887BC
:10134000EDCF10E076CFFC019085957081E095306F
:1013500009F080E00895CF92DF92EF92FF920F9311
:101360001F93CF93DF93EC0188858B7F8887E8817B
:10137000F9810190F081E02DCE010995182F888523
:10138000869581701817B9F00E94A4086A837B8340
:101390008C839D83888592E089278887888582FB56
:1013A000882780F9DF91CF911F910F91FF90EF90E7
:1013B000DF90CF9008950E94A408CA80DB80EC8063
:1013C000FD80AB01BC014C195D096E097F098E815E
:1013D0009F81B0E0A0E0481759076A077B07F0F249
:1013E000888581701817D1F20E94A4086A837B83D4
:1013F0008C839D83888591E08927846088870E94FB
:10140000A40809851A852B853C85601B710B820B0E
:10141000930B6D877E878F87988B0E94A4086987BE
:101420007A878B879C87BACFCF93DF93EC0118869E
:10143000E881F9810190F081E02D0995882319F068
:101440008885836088870E94A4086A837B838C8355
:101450009D83DF91CF910895862FBA010C940B07DD
:10146000FC01818930E020E08B3218F40E94FE07F5
:101470009C0181E0232B09F480E008950895EF9208
:10148000FF920F931F93CF93DF937C01EB018B01AE
:10149000040F151FC017D10759F0D701ED91FC912A
:1014A0000480F581E02D6881C70109958993F2CF09
:1014B000DF91CF911F910F91FF90EF9008950F93BF
:1014C0001F93CF93DF93EC018B018091C008E881DB
:1014D000F9810480F581E02D86FD13C0612FCE01D6
:1014E0000995182FE881F9810480F581E02D602F9E
:1014F000CE010995082FC801DF91CF911F910F915F
:101500000895CE010995082FE881F9810480F581BD
:10151000E02D612FCE010995182FEDCF00006093CB
:10152000C4088091C30887FFFCCF8091C408089548
:101530008F929F92AF92BF92CF92DF92EF92FF92E3
:101540000F931F93CF93DF93FC018085882319F0BD
:1015500081FF0EC07894DF91CF911F910F91FF9082
:10156000EF90DF90CF90BF90AF909F908F900895B5
:1015700080FFF1CF82849384A484B584C12CD12CC4
:10158000760110E09401A501B601C701A0E00E9418
:101590008B5599F1217030E040E050E060E070E060
:1015A00080E090E00E948B55D9F0D0E0C0E010338D
:1015B00070F4C12FC695C695C69580E2C89FE0011C
:1015C0001124C05FDB4F812F8770C80FD11DCF0161
:1015D000810F911DDC0152968C919881892B888313
:1015E0009401A501B601C70101E00E9470554901AF
:1015F0005A016B017C011F5FC5CF86849784A08848
:10160000B188C12CD12C760110E29401A501B6015C
:10161000C701A0E00E948B5509F49DCF217030E0F6
:1016200040E050E060E070E080E090E00E948B5588
:10163000D9F0D0E0C0E0103370F4C12FC695C69544
:10164000C695B0E2CB9FE0011124C05FDB4F812F34
:101650008770C80FD11DCF01810F911DDC015296FB
:101660008C919881892B88839401A501B601C701CB
:1016700001E00E94705549015A016B017C011F5F16
:10168000C4CFFC016F3F710581F1808581FD2DC0C4
:10169000603271055CF581E090E002C0880F991F0F
:1016A0006A95E2F780959095092E000CAA0BBB0B6A
:1016B000428553856485758584239523A623B723A6
:1016C00082879387A487B58782859385A485B5850E
:1016D000892B8A2B8B2B49F486859785A089B18924
:1016E000892B8A2B8B2B09F410860895605271097F
:1016F00081E090E002C0880F991F6A95E2F780951B
:101700009095092E000CAA0BBB0B46855785608966
:10171000718984239523A623B72386879787A08B77
:10172000B18BD2CFFC016F3F7105E9F160337105D8
:101730001CF082E080870895808581608087603218
:101740007105C4F481E090E002C0880F991F6A958A
:10175000E2F7092E000CAA0BBB0B4285538564856A
:101760007585842B952BA62BB72B82879387A4870F
:10177000B58708956052710981E090E002C0880F3A
:10178000991F6A95E2F7092E000CAA0BBB0B468540
:10179000578560897189842B952BA62BB72B86875B
:1017A0009787A08BB18B0895E0ECF8E020812E7F25
:1017B0002083FC0117820895E0ECF8E082818E7F9F
:1017C00082830895E0ECF8E082818160828308954D
:1017D0000F9391E09093422A1092412A60933F2AFE
:1017E0007093402A40933E2A20933D2A10923C2A2F
:1017F00010923B2A00933A2A880F8093392A23E0DB
:1018000030E044E050E080913E2A882341F020936C
:10181000372A3093382A8091392A8E7F0BC08091E5
:101820003D2A882351F04093372A5093382A8091DB
:10183000392A81608093A70808C080913E2A8111CF
:1018400004C080913D2A882311F38091412A882386
:10185000E1F38091412A8330B1F280913D2A8823BF
:1018600021F080913B2A0F9108958091412A823086
:1018700031F0853031F0813031F480E0F4CF81E017
:10188000F2CF83E0F0CF84E0EECFE0EAF8E091859C
:101890009066918722E030E02093372A3093382AEF
:1018A0008093292A1092282A089581E08093282A7B
:1018B0001092292A93E09093AA089091AB0891FF87
:1018C00010C01092352AE091262AF091272A099516
:1018D0008093342A85E090E08093372A9093382AC9
:1018E00008951092362A8093332A86E090E0F4CF50
:1018F0008F929F92AF92BF92CF92DF92EF92FF9220
:10190000CF93DF9360342DE0720723E082079105C7
:1019100008F454C0611525E372072CE08207910595
:1019200008F445C060387F448241910508F046C004
:10193000C8E7D0E020E432E44FE050E08090112886
:1019400090901228A0901328B0901428C501B401DB
:101950000E94C75069017A018AE0C81AD108E108DB
:10196000F108C501B40120E432E44FE050E00E94E8
:10197000C750DE010E94835028EE33E040E050E083
:101980000E94C750C21AD30AE40AF50AF694E794F3
:10199000D794C794C092A608DF91CF91FF90EF90A3
:1019A000DF90CF90BF90AF909F908F900895CCE242
:1019B000D1E020E83AE146E050E0C0CFC8EED3E005
:1019C00020EA36E841E050E0B9CF6093242A7093D2
:1019D000252A08956093222A7093232A0895E0917E
:1019E000242AF091252A309741F01092212A109252
:1019F000202A09958091202A089580E00895E09199
:101A0000222AF091232A309759F030911F2A2091F1
:101A10001E2A321728F010921F2A80931E2A09943A
:101A200008950895E0911F2A80911E2AE81730F446
:101A3000F0E0E256F64D808190E008958FEF9FEF41
:101A4000089590911F2A80911E2A2FEF3FEF98173B
:101A500048F4E92FF0E0E256F64D208130E09F5F38
:101A600090931F2AC901089580911E2A90911F2AE0
:101A7000891B990B0895CF92DF92EF92FF920F93FB
:101A80001F93CF93DF937C018A01EB016B01C40E9E
:101A9000D51ECC15DD0551F06991D701ED91FC9172
:101AA0000190F081E02DC7010995F3CFC801DF91C6
:101AB000CF911F910F91FF90EF90DF90CF900895FD
:101AC0002091202A27FF08C021E030E0FC0122837A
:101AD000338390E080E008958091212AE82FF0E0A0
:101AE000E25EF64D60838F5F8093212A8093202AE7
:101AF00081E090E00895DC01ED91FC91008CF18D86
:101B0000E02D61E009940F938091372A9091382A53
:101B10000197A1F48091422A811112C0062F20E082
:101B20004091202A6EE179E280911D290E94E80B04
:101B30001092212A1092202A0F91089580E0F8CF68
:101B400081E0F6CF60931D291092212A1092202A5D
:101B50000895DC01ED91FC91048CF58DE02D21E0E0
:101B600009940F938EE999E280932A2A90932B2A65
:101B70008091372A9091382A0197C9F48091422A9E
:101B8000811117C0FA014138510510F0E0E8F0E08A
:101B9000022F862F2E2F40E070E060E00E94E80BBD
:101BA00010921F2A80931E2A90E00F91089580E0E2
:101BB000F7CF81E0F5CFCB01BA010C94780CE0EAC5
:101BC000F8E01382168281E08583148611861092D4
:101BD000372A1092382A089510921F2A10921E2A2E
:101BE0001092212A1092202A8091372A9091382A27
:101BF000892BD9F482E090E08093372A9093382A99
:101C00001092362A1092352A1092282A1092292AE8
:101C100010921C291092332A660F6093AC0881EE53
:101C20008093A90881E08093A3088FEE9CE08093C5
:101C3000262A9093272A8EE199E280932C2A90936A
:101C40002D2A8FEF9CE08093312A9093322A8EE9DF
:101C500099E280932E2A90932F2A80E88093302A4D
:101C6000089510921F2A10921E2A1092212A109273
:101C7000202A8091372A9091382A892B41F562E0F9
:101C800070E086E10E94D20662E070E087E10E9487
:101C9000D2068091E3058093E30581E090E0809394
:101CA000372A9093382A10923B2A10923C2A10929D
:101CB000422A1092412A81EC8093A30860EA76E8D8
:101CC00081E090E00E94780C81E08093A50808955F
:101CD000FC01A5A1B6A18C9192A589238C93A5A105
:101CE000B6A18C9191A5892B8C930895DC019396D4
:101CF000ED91FC919497908198968C9189238083A3
:101D00000895DC019396ED91FC91949790819796BC
:101D10008C91892B80830895DC019196ED91FC9143
:101D20009297908196968C91892380830895DC0107
:101D30009196ED91FC919297908195968C91892B3B
:101D400080830895CF92DF92EF92FF921F93CF93FB
:101D5000DF93EC016A017B018DA981112BC08F2DCE
:101D60009927AA27BB278093C4088091C30887FFBF
:101D7000FCCFC701AA27BB278093C4088091C30862
:101D800087FFFCCFBB27AF2D9E2D8D2D8093C408E0
:101D90008091C30887FFFCCFC092C4088091C3081C
:101DA00087FFFCCFDF91CF911F91FF90EF90DF90E5
:101DB000CF9008958130B1F410E2CE01F7FE0FC04C
:101DC0000E94970ECE010E94810ECE010E94760ED7
:101DD000CC0CDD1CEE1CFF1C115079F7E3CF0E94E8
:101DE0008C0EF0CFEF8DF8A18F2D9927AA27BB2756
:101DF0008083CE010E94680EEF8DF8A1C701AA274B
:101E0000BB278083CE010E94680EEF8DF8A1BB270F
:101E1000AF2D9E2D8D2D8083CE010E94680EEF8DFB
:101E2000F8A1C082CE01DF91CF911F91FF90EF907A
:101E3000DF90CF900C94680EFF920F931F93CF9377
:101E4000DF93EC018B018DA9811112C01093C4089E
:101E50008091C30887FFFCCF0093C4088091C3081A
:101E600087FFFCCFDF91CF911F910F91FF900895D5
:101E70008130B1F490E1F92ECE0117FF0EC00E941F
:101E8000970ECE010E94810ECE010E94760E000FA9
:101E9000111FFA94F110F0CFE5CF0E948C0EF1CF14
:101EA000EF8DF8A11083CE010E94680EEF8DF8A18E
:101EB0000083CE01DF91CF911F910F91FF900C9481
:101EC000680E0F931F93CF93DF93EC01162F8DA90C
:101ED00081110BC06093C4088091C30887FFFCCFB9
:101EE000DF91CF911F910F910895813099F408E00F
:101EF000CE0117FF0CC00E94970ECE010E94810EEA
:101F0000110FCE010E94760E015091F7E9CF0E9489
:101F10008C0EF3CFEF8DF8A16083CE01DF91CF91CE
:101F20001F910F910C94680ECF93DF93EC01ED8D10
:101F3000FE8D80819CA989238083CE010E94610F40
:101F4000ED8DFE8D80819BA9892B8083DF91CF91C0
:101F500008958F929F92AF92BF92CF92DF92EF92AD
:101F6000FF920F931F93CF93DF93EC0189AD9AAD4E
:101F7000680F791F8BAD9CAD480F591F2150310957
:101F8000260F371F4901B12CA12CCB01B0E0A0E0F6
:101F9000DC0199278827882A992AAA2ABB2A68015E
:101FA00081E0C81AD108C40ED51EF12CE12C70E0D6
:101FB00060E0BA0155274427C42AD52AE62AF72A21
:101FC0006AE2CE010E94940FB501A401CE010E94E5
:101FD000A20E6BE2CE010E94940FB701A601CE01C2
:101FE0000E94A20E6CE2CE01DF91CF911F910F9162
:101FF000FF90EF90DF90CF90BF90AF909F908F9029
:102000000C94940FDC01D5962C91D59721110AC020
:102010005F968D919C91DC01ED91FC910088F18996
:10202000E02D099408950F931F93CF93DF93EC0154
:102030002DA9211121C0DC018F8D98A1EC01E8812F
:10204000F9810684F785E02D91960C9191979296EF
:102050001C91929793962C91939794963C91949778
:1020600095964C91959796965C91969797966C91CC
:10207000979798967C910995DF91CF911F910F9139
:1020800008950F931F93CF93DF93EC018B010E9470
:1020900013108FA987FD06C0EB8DFC8D80819AA956
:1020A00089238083ED8DFE8D80819CA98923808387
:1020B00066E3CE010E94610FED8DFE8D80819BA9AC
:1020C000892B80838DA9F8018230A1F06081CE0137
:1020D0000E94610F8FA987FD06C0EB8DFC8D80816A
:1020E00099A9892B8083CE01DF91CF911F910F9108
:1020F0000C94021088A9882349F360817181CE0174
:102100000E941C0FE7CFCF93DF931F92CDB7DEB7AE
:10211000FC0119826370668BDC01AD5BBF4F2C91B3
:1021200030E011968C9190E0623031F06330C9F06C
:10213000613081F040EC498321AF32AF83AF94AF7F
:10214000BE016F5F7F4FCF010E9441100F90DF9162
:10215000CF91089540EA498323AF34AF81AF92AF66
:10216000EFCF40E6F8CF0F931F93CF93DF931F92EB
:10217000CDB7DEB7FC0119826370668BDC01A85B0A
:10218000BF4F2D913C91119712968D919C91623089
:10219000D1F1633009F440C08F010C5B1F4F6130F7
:1021A000F9F040EC4983AF014D5B5F4FDA014C9190
:1021B00050E041AF52AFD8014C9150E043AF54AF23
:1021C0002087318782879387BE016F5F7F4FCF0162
:1021D0000E9441100F90DF91CF911F910F910895B0
:1021E00040EA4983D8014C9150E041AF52AFDF0142
:1021F000AA5BBF4F4C9150E043AF54AF2287338767
:1022000080879187E1CFDF01AA5BBF4F4C9150E0FF
:1022100041AF52AF1196D0CF40E64983DF01A95BB1
:10222000BF4F4C9150E041AF52AF1497E3CF1F9393
:10223000CF93DF93EC01162FE881F9810284F385B7
:10224000E02D0995112371F06DADCE010E94940F20
:10225000E881F9810688F789E02DCE01DF91CF91E1
:102260001F9109946EADF1CFAF92BF92CF92DF92E2
:10227000EF92FF920F931F93CF93DF93EC0177FDC3
:1022800038C088859985681779079CF557FD31C056
:102290008A859B854817590764F569017A015B01B6
:1022A000E881F9810284F385E02DCE010995E8816A
:1022B000F98102A4F3A5E02D01E010E021E030E077
:1022C000A701B501CE010995B601CE010E941C0FF0
:1022D000E881F9810688F789E02DCE01DF91CF9161
:1022E0001F910F91FF90EF90DF90CF90BF90AF9034
:1022F0000994DF91CF911F910F91FF90EF90DF90A4
:10230000CF90BF90AF9008958F929F92AF92BF925F
:10231000CF92DF92EF92FF920F931F93CF93DF93B1
:10232000EC0149015701E881F98102A4F3A5E02DF0
:1023300009959401D8010E945F556B017C01C1147D
:10234000D104E104F10409F481C08DA9811119C0FF
:1023500081E0C81AD108E108F1088FEFC816D80645
:10236000E806F80609F472C0B092C4088091C30868
:1023700087FFFCCFA092C4088091C30887FFFCCFE1
:10238000E7CF813099F581E0C81AD108E108F1085A
:102390008FEFC816D806E806F80609F457C00B2DCB
:1023A00018E0CE0107FF1CC00E94970ECE010E94CC
:1023B000810ECE010E94760E000F115091F70A2D6A
:1023C00018E0CE0107FF0FC00E94970ECE010E94B9
:1023D000810ECE010E94760E000F115091F7D3CFDF
:1023E0000E948C0EE3CF0E948C0EF0CFBA1016C064
:1023F000CC0CDD1CEE1CFF1CEF8DF8A1B08281E03F
:10240000C81AD108E108F1088FEFC816D806E80607
:10241000F806E1F0CE010E94680EF1CF81E0C81A03
:10242000D108E108F1088FEFC816D806E806F806CB
:1024300069F0EF8DF8A1B082CE010E94680EEF8D99
:10244000F8A1A082CE010E94680EE8CFDF91CF9163
:102450001F910F91FF90EF90DF90CF90BF90AF90C2
:102460009F908F9008958F929F92AF92BF92CF923C
:10247000DF92EF92FF920F931F93CF93DF934C0164
:10248000EB016A01590137FF07C0C9010196C80F66
:10249000D91FB194A194B108F401A085B185CA17E0
:1024A000DB070CF058C017FF07C0C8010196C80E23
:1024B000D91E119501951109F40182859385C816DD
:1024C000D9060CF048C0FE01EA0DFB1DAF014150DA
:1024D000510957FD40C0B601600F711F9B0121508B
:1024E000310937FD38C0D7FF03C05F01D0E0C0E03D
:1024F000D7FE03C08B01D12CC12C4A175B071CF0FF
:102500005D01AC1ABD0A281739071CF08C010C19A3
:102510001D09D401ED91FC910284F385E02DC401E5
:1025200009959501A601BE01C4010E948411D40140
:10253000ED91FC910688F789E02DC401DF91CF91E0
:102540001F910F91FF90EF90DF90CF90BF90AF90D1
:102550009F908F900994DF91CF911F910F91FF90E1
:10256000EF90DF90CF90BF90AF909F908F900895A5
:10257000EF92FF920F931F932115310529F001155A
:10258000110511F00E9433121F910F91FF90EF90EF
:1025900008958F929F92AF92BF92CF92DF92EF9267
:1025A000FF920F931F93CF93DF935C014B016A015E
:1025B000E90177FD52C0DC0118968D919C91681756
:1025C00079070CF04AC0209709F447C037FF07C0CD
:1025D000C9010196C80ED91ED195C195D109F50141
:1025E00082859385C816D906C4F5A6014C0F5D1FD8
:1025F0009A012150310937FD30C0D7FE03C0EA01EE
:10260000D12CC12C281739071CF0EC01CC19DD099D
:10261000D501ED91FC910284F385E02DC50109956A
:1026200078018E0121E030E0A601B401C5010E94CD
:102630008411D501ED91FC910688F789E02DC50143
:10264000DF91CF911F910F91FF90EF90DF90CF908E
:10265000BF90AF909F908F900994DF91CF911F9181
:102660000F91FF90EF90DF90CF90BF90AF909F9031
:102670008F9008958F929F92AF92BF92CF92DF92E8
:10268000EF92FF920F931F93CF93DF935C016B0147
:102690004A01E90157FD52C0DC011A968D919C91C7
:1026A000481759070CF04AC0209709F447C037FF74
:1026B00007C0C9010196C80ED91ED195C195D1098F
:1026C000F50180859185C816D906C4F5A6014C0F81
:1026D0005D1F9A012150310937FD30C0D7FE03C07C
:1026E000EA01D12CC12C281739071CF0EC01CC19B8
:1026F000DD09D501ED91FC910284F385E02DC50142
:102700000995780101E010E09E01A401B601C50120
:102710000E948411D501ED91FC910688F789E02D86
:10272000C501DF91CF911F910F91FF90EF90DF9046
:10273000CF90BF90AF909F908F900994DF91CF91F1
:102740001F910F91FF90EF90DF90CF90BF90AF90CF
:102750009F908F900895EF92FF920F931F93CF93C6
:10276000DF9377FD32C0DC011896ED91FC916E1776
:102770007F075CF52115310541F137FF07C0F901ED
:1027800031964E0F5F1F319521953109DC011A9664
:10279000ED91FC914E175F07C4F4EA01C20FD31FFD
:1027A000DE011197B7FD11C057FF03C09E0150E035
:1027B00040E0AE17BF071CF09F01241B350B7801CA
:1027C000890121E030E00E948411DF91CF911F91B7
:1027D0000F91FF90EF900895EF92FF920F931F9348
:1027E000CF93DF9357FD31C0DC011A96ED91FC9138
:1027F0004E175F0754F52115310539F137FF07C032
:10280000F90131966E0F7F1F319521953109DC0159
:102810001896ED91FC916E177F07BCF4EB01C20F87
:10282000D31FDE011197B7FD10C077FF03C09E01D3
:1028300070E060E0AE17BF071CF09F01261B370B4E
:10284000780101E010E00E948411DF91CF911F9187
:102850000F91FF90EF9008958F929F92AF92BF9249
:10286000CF92DF92EF92FF920F931F93CF93DF935C
:1028700047012115310509F44BC00115110509F473
:1028800047C037FF07C0F90131966E0F7F1F3195A2
:1028900021953109DC011896AD90BC906A157B0535
:1028A000BCF517FF07C0F80131964E0F5F1F119559
:1028B00001951109DC011A96ED91FC914E175F0705
:1028C0003CF56B01C20ED31EE6012197D7FD20C057
:1028D0007A01E00EF11ED7011197B7FD19C077FFFD
:1028E00003C0960170E060E057FF03C0870150E02D
:1028F00040E0CA15DB051CF09501261B370BAE170F
:10290000BF071CF08F01041B150B74010E9484117A
:10291000DF91CF911F910F91FF90EF90DF90CF90BB
:10292000BF90AF909F908F900895EF92FF920F937A
:102930001F93CF93DF93EC0177FD22C088859985A3
:1029400068177907ECF457FD1BC08A859B854817EB
:102950005907B4F47901E881F98102A4F3A5E02DC7
:1029600001E010E021E030E0CE010995B701CE0191
:10297000DF91CF911F910F91FF90EF900C941C0F5E
:10298000DF91CF911F910F91FF90EF900895DC019F
:10299000D7962C91D79727FD09C05B96ED91FC91B6
:1029A0005C972081D1963C91232B20830C940210BC
:1029B000CF93DF93EC010E9413108FA987FD06C00F
:1029C000EB8DFC8D80819AA989238083DF91CF9143
:1029D00008950895FC016370668B8481958126813A
:1029E0003781613039F0633029F080879187228701
:1029F00033870895208731878287938708952F92A0
:102A00003F924F925F926F927F928F929F92AF927E
:102A1000BF92CF92DF92EF92FF920F931F93CF93CB
:102A2000DF93CDB7DEB76A97CDBFDEBF898F9A8FB0
:102A300069837A834A01D22E0F8318873701BC2C11
:102A4000DC0159962D913C915A972115310509F0D9
:102A500012C118968D919C911997681779070CF0FF
:102A6000D4C11A968D919C91481759070CF0CDC18D
:102A70004C2C512CB6E0CB9E600D711D11246B8740
:102A80007C87161617060CF0C0C1EA2DF0E0E98726
:102A9000FA8793E0EE0FFF1F9A95E1F7EF87F88B27
:102AA000CF01840F951F181619060CF0AEC1A98D21
:102AB000BA8D58968C91811104C0BFEABD1508F4F7
:102AC000D394A98DBA8DED91FC9111970284F38571
:102AD000E02DCD010995B5E0DB9EC0011124E9810F
:102AE000FA81EB83FC83312C212C9C0128513D4F32
:102AF0002F8B388F4A2D50E04D8B5E8BEF89F88DF0
:102B0000E20DF31D44918D829E82D12CC12C6981EE
:102B10007A81620D731D698B7A8B842F90E08B8B89
:102B20009C8BE98DFA8DA081B18140FF7FC0F1E0DF
:102B3000BF126CC0AF126AC01C96ED91FC912F8140
:102B40003885A4014C0D5D1D69897A89898D9A8D1E
:102B50000995EB89FC89F595E7954E2F5FEFC51A2E
:102B6000D50A6D817E818D899E89680F791F6D835D
:102B70007E8398E0C916D10481F6AFEF2A1A3A0A8B
:102B8000EB81FC81E40DF51DEB83FC83F5E02F1652
:102B9000310409F0B3CF2F81388526153705B9F0F8
:102BA000A98DBA8DED91FC91B1E0BB1254C0AB126E
:102BB00052C069817A816B5F7F4F0088F189E02D77
:102BC000830128E030E0A401898D9A8D0995A98DB3
:102BD000BA8DED91FC9111970688F789E02DCD0112
:102BE0006A96CDBFDEBFDF91CF911F910F91FF900D
:102BF000EF90DF90CF90BF90AF909F908F907F909D
:102C00006F905F904F903F902F9009941E96ED919A
:102C1000FC91EF80F88409851A8592014D815E81CF
:102C20006B817C81898D9A8D099593CF2F81388511
:102C30002615370509F48DCF31E0B31207C0A31272
:102C400005C01C96ED91FC9193017BCF1E96ED91F2
:102C5000FC917301E0CF6B857C856419750906844E
:102C6000F785E02D73010F8518899201A401898DE4
:102C70009A8D0995ACCFF90134969491329745918C
:102C80005491D91AB7E0DB9E400D511D1124F90172
:102C9000259134912B8B3C8BFA0125903490FA01CD
:102CA0003296749031963491398B32966490319685
:102CB000449041E04C1518F04A1508F07FC0662D8D
:102CC000062C000C770B6B837C83842D042C000C6A
:102CD000990B8D839E83A98DBA8DED91FC911197EF
:102CE0000284F385E02DCD010995512CD12CC12C06
:102CF000EA2DF0E0E987FA872B2D30E02B873C871F
:102D0000A401440D511D47FC5A954F8B588F698182
:102D10007A81660D711D67FC7A956D877E8779894A
:102D2000C71608F054CF2C2D30E04D815E81420F44
:102D3000531FA985BA854A9FC0014B9F900D5A9F8A
:102D4000900D1124FC01E80DF91DEF87F88B852DFE
:102D5000612C4F89588D420F531F4D8B5E8B67142A
:102D600008F050C044244394480E877041F4C101D8
:102D70000196EB89FC89E20DF31DD4901C01D7FE6E
:102D800019C0A98DBA8DED91FC91662D70E0B1E06E
:102D9000BB1219C0AB1217C02D853E85620F731F81
:102DA0000484F585E02D2F8138854D895E89898DD4
:102DB0009A8D0995DD0C6394842DD1CF1D821E82DE
:102DC0001B821C8288CF4B815C81640F751FAB8591
:102DD000BC856A9FC0016B9F900D7A9F900D112456
:102DE00069817A81680F791F0684F785E02DEF806D
:102DF000F88409851A859D014F855889898D9A8D9A
:102E00000995D8CF570CC3948ACF6A96CDBFDEBF41
:102E1000DF91CF911F910F91FF90EF90DF90CF90B6
:102E2000BF90AF909F908F907F906F905F904F90EA
:102E30003F902F9008958F929F92AF92CF92EF92F2
:102E4000FF920F931F93CF93DF93EC01262F898D71
:102E50009A8D009709F051C06A30D1F41C861D8606
:102E60008D8948E0849F900111248E859F85820F73
:102E7000931F8E879F8781E090E0DF91CF911F9114
:102E80000F91FF90EF90CF90AF909F908F9008950B
:102E90006D3089F3CC88AD888F898823C1F08C850B
:102EA0009D8536E0C39E800D911D1124488559856E
:102EB0004817590764F44E855F851C861D8638E0E7
:102EC000A39EC0011124840F951F8E879F87EA88D7
:102ED000FB88088919894E855F856C857D85CE01C3
:102EE0000E94FF142C898C859D8546E0249F800DCF
:102EF000911D11248C879D87BECF6A3069F41C8692
:102F00001D86FC013896E4912D898E859F85E29F70
:102F1000800D911D1124ADCF6D3009F4ACCFFC01B3
:102F200034963491631708F4A6CF3296E491E617ED
:102F300008F4A1CFFC01329685909490462F431B54
:102F4000342F47E0349F800C911C1124F4013296F9
:102F500034913196E4913323A9F1EE2399F1CC8891
:102F6000F4013596E491AD884F89442301F10E2E8A
:102F7000000CFF0BE30FF11DCE9EA001CF9E500D64
:102F800011246C857D85460F571F688579856417E8
:102F900075076CF44E855F851C861D86FC0138968E
:102FA000E491AE9E400D511D11244E875F87EA8843
:102FB000FB88088919894E855F856C857D85CE01E2
:102FC0000E94FF14F4013496E4912C898C859D8530
:102FD000E29F800D911D11248DCF6F927F928F9271
:102FE0009F92AF92BF92CF92DF92EF92FF920F9398
:102FF0001F93CF93DF93EC016B015A013901480114
:10300000E881F9810284F385E02D0995E881F98151
:103010000288F389E02D87019301A501B601CE0155
:103020000995A501480D591D41505109E881F981C3
:103030000288F389E02D9301B601CE010995E8815C
:10304000F9810088F189E02D9401A501B601CE0136
:103050000995C60CD71CB60161507109E881F98148
:103060000088F189E02D9401A501CE010995E88140
:10307000F9810688F789E02DCE01DF91CF911F916C
:103080000F91FF90EF90DF90CF90BF90AF909F9007
:103090008F907F906F9009946F927F928F929F9202
:1030A000AF92BF92CF92DF92EF92FF920F931F9356
:1030B000CF93DF935C01EB016A014901380187017D
:1030C000DC01ED91FC916217730719F56416750622
:1030D0002CF0962D872D3A01C92ED82E960126194F
:1030E00037092F5F3F4F048CF58DE02DA301BE0102
:1030F000C5010995DF91CF911F910F91FF90EF903E
:10310000DF90CF90BF90AF909F908F907F906F9007
:1031100008954615570591F42617370724F0892D91
:103120004B01C22FD82F9E01281939092F5F3F4F1D
:10313000068CF78DE02DA601B401DACF0284F38569
:10314000E02D0995D501ED91FC910488F589E02DDC
:1031500083019401A601BE01C5010995D501ED9138
:10316000FC910688F789E02DC501DF91CF911F9171
:103170000F91FF90EF90DF90CF90BF90AF909F9016
:103180008F907F906F900994EF92FF920F931F930F
:10319000DC011A960D911C911B9718962D913C916C
:1031A0001997ED91FC9100A0F1A1E02D7B0150E079
:1031B00040E070E060E009951F910F91FF90EF9063
:1031C00008954F925F926F927F928F929F92AF92EB
:1031D000BF92CF92DF92EF92FF920F931F93CF9304
:1031E000DF936C012B015A0139014801DC01ED919B
:1031F000FC910284F385E02D0995E201640C751CB5
:10320000D601ED91FC91C615D7055CF40088F189D3
:10321000E02D87019401A501BE01C6010995219603
:10322000EFCF0688F789E02DC601DF91CF911F917E
:103230000F91FF90EF90DF90CF90BF90AF909F9055
:103240008F907F906F905F904F9009948F929F9294
:10325000AF92BF92CF92DF92EF92FF920F931F93A4
:10326000CF93DF93EC015B014A016901E881F981A9
:103270000284F385E02D099595012C0D3D1D21500B
:103280003109E881F9810488F589E02D780184010C
:10329000A401B501CE010995E881F9810688F78975
:1032A000E02DCE01DF91CF911F910F91FF90EF9014
:1032B000DF90CF90BF90AF909F908F9009948F92A6
:1032C0009F92AF92BF92CF92DF92EF92FF920F93B5
:1032D0001F93CF93DF93EC015B014A0169017801F1
:1032E000E881F9810284F385E02D0995C80CD91C89
:1032F000860101501109E881F9810488F589E02DE2
:103300009501A401B501CE010995E881F9810688EE
:10331000F789E02DCE01DF91CF911F910F91FF90A2
:10332000EF90DF90CF90BF90AF909F908F900994D7
:10333000EF92FF920F931F93DC01ED91FC9100A09F
:10334000F1A1E02D09951F910F91FF90EF90089545
:103350000F931F93DC01ED91FC91068CF78DE02D0E
:1033600009951F910F9108950F931F93DC01ED9123
:10337000FC91048CF58DE02D09951F910F91089516
:10338000DC01ED91FC910084F185E02D09942F92F0
:103390003F924F925F926F927F928F929F92AF92E5
:1033A000BF92CF92DF92EF92FF920F931F93CF9332
:1033B000DF93CDB7DEB72697CDBFDEBF3C016A01F4
:1033C0002D833E83EB82FC825801A41AB50AB7FE16
:1033D00003C0B194A194B1088D809E80861A970A8B
:1033E00097FE03C09194819491088A149B045CF029
:1033F000902F812F0D811E819D838E839C2D8D2D7D
:103400006B01692F782F0C151D055CF09D818E8155
:103410006D837E83692F782F902F812F8601C92E8F
:10342000D82E1601201A310A2B012D813E81421A15
:10343000530A57FE03C0519441945108710137FE5D
:1034400003C03FEFE31AF30AF594E7948D819E8160
:10345000861797075CF5A1E0B0E0A983BA83C01690
:10346000D1064CF1D301ED91FC910484F585E02D5A
:103470002B813C81A8016D817E818A149B041CF004
:103480004D815E81B801C3010995E418F508F7FE86
:103490000AC02D813E8189819A81280F391F2D8391
:1034A0003E83E20CF31C0F5F1F4FD9CF2FEF3FEF8E
:1034B00029833A83D4CF2696CDBFDEBFDF91CF914B
:1034C0001F910F91FF90EF90DF90CF90BF90AF9042
:1034D0009F908F907F906F905F904F903F902F9034
:1034E0000895089590E080E00895DC015A96ED91EA
:1034F000FC91309709F009940895DC015896ED91FC
:10350000FC91309709F009940895DC015696ED91ED
:10351000FC91309709F009940895DC015496ED91DF
:10352000FC91309709F009940895362F642FDC013F
:103530001E96ED91FC91309719F0422F832F09943C
:103540000895DC01ED91FC910088F189E02D23E0E4
:1035500030E00994CF92DF92EF92FF920F931F9386
:10356000CF93DF93FC01278130852250310922302F
:10357000310530F58C010E94A408F801C785D08977
:103580000385148525853685601B710B820B930B93
:103590009E010D2E000C440B550B0E94C750AE012E
:1035A000D7FF02C04F5F5F4F559547956A01550F92
:1035B000EE08FF0821E0C616D706E806F90608F06F
:1035C00020E0822FDF91CF911F910F91FF90EF901C
:1035D000DF90CF900895862F9091B12A9923A1F082
:1035E0006CE00E943955E92FF0E0EE0FFF1FE85123
:1035F000F2418081918197FD07C080933528909397
:10360000362881E08093B32A0895FC01208131811E
:1036100042815381FB0160817181828193810E948B
:10362000F8500E94DC51CB010895CF92DF92EF92C7
:10363000FF920F931F93CF93DF936C019A018BE15D
:10364000869FE001879FD00D1124F12CE12C0BE126
:1036500010E0AE01B6018BEB9DE20E94B812EBEBDD
:10366000FDE2C486D5862396C687D787DF91CF91A2
:103670001F910F91FF90EF90DF90CF9008951092DF
:103680000D2910920E2910920F29109210291092D4
:10369000CF2A1092D02A10923828109239281092EE
:1036A0003A2810923B281092092910920A29109268
:1036B00007291092082908954F925F926F927F9286
:1036C0008F929F92AF92BF92CF92DF92EF92FF9232
:1036D0000F931F93CF93DF93CDB7DEB72E97CDBF58
:1036E000DEBF8091452890914628029709F04FC18E
:1036F0002091E32A298381E082278093D22A0E94A5
:1037000045084B015C013981332309F438C18091AC
:10371000A2289091A328A091A428B091A528A50142
:103720009401281B390B4A0B5B0BCA01B9010E949B
:10373000125269837A838B839C8320913128309144
:10374000322840913328509134280E94215320E0A0
:1037500030E044EB52E40E946A5120E030E040E067
:103760005FE30E94F9500E94DC516B01770FEE0875
:10377000FF080091442C1091452CD8018C918E7F2C
:103780008C938C918670823009F45FC0843051F044
:1037900081110FC044E0CC0CDD1CEE1CFF1C4A95CF
:1037A000D1F707C062E0F694E794D794C7946A957E
:1037B000D1F780E090E0A1E0B0E08093522C9093AC
:1037C000532CA093542CB093552C97014427552784
:1037D0002B873C874D875E872093462C3093472C60
:1037E0004093482C5093492CC701B601882799274C
:1037F00060934A2C70934B2C80934C2C90934D2CBF
:10380000232B242B252B09F444C0412C512C3201AD
:103810006394A301920121503109410951092D837B
:103820003E834F8358876130710581059105A9F466
:10383000C701B6010E94C7502B873C874D875E8722
:103840004D805E806F807884E4CF53E0CC0CDD1C2B
:10385000EE1CFF1C5A95D1F7ACCF60934A2C7093A5
:103860004B2C80934C2C90934D2C4092522C509288
:10387000532C6092542C7092552C2B853C854D8591
:103880005E852093462C3093472C4093482C5093D0
:10389000492C8091522C9091532CA091542CB09192
:1038A000552C0197A109B1098093522C9093532C68
:1038B000A093542CB093552C40914A2C50914B2CF2
:1038C00060914C2C70914D2C41155105610571058D
:1038D00061F0415051096109710940934A2C50939C
:1038E0004B2C60934C2C70934D2C4091462C509156
:1038F000472C6091482C7091492C40934E2C50934A
:103900004F2C6093502C7093512C452B462B472BFA
:1039100021F480914A2C90914B2CD8011C968D93C8
:103920009C931D971A961D921C921B978C918160F7
:103930008C93C501B4010E9412526B017C0120E0FE
:1039400030E040EC5FE369817A818B819C810E9449
:1039500021539B01AC01C701B6010E94F95020E040
:1039600030E04AE754E40E946A510E94E3516093B8
:10397000DF2A7093E02A8093E12A9093E22A8092D2
:10398000A2289092A328A092A428B092A5282E96AF
:10399000CDBFDEBFDF91CF911F910F91FF90EF90D0
:1039A000DF90CF90BF90AF909F908F907F906F905F
:1039B0005F904F9008958091452890914628892BDB
:1039C00029F08091E32A882309F454C08091582A71
:1039D0009091592AA0915A2AB0915B2A0196A11D73
:1039E000B11D8093582A9093592AA0935A2AB093D4
:1039F0005B2A80911628909117284091582A50915F
:103A0000592A60915A2A70915B2A092E000CAA0B40
:103A1000BB0B481759076A077B0748F081E090E025
:103A20008093D52A9093D62A8093D32A08958091A3
:103A30001628909117284091582A5091592A609140
:103A40005A2A70915B2A97FD019695958795092EC4
:103A5000000CAA0BBB0B481759076A077B0750F0ED
:103A60008091D52A9091D62A892B21F01092D52ABF
:103A70001092D62A08954F925F926F927F928F9202
:103A80009F92AF92BF92CF92DF92EF92FF92CF932D
:103A9000DF93EC016A017B01488459846A847B844A
:103AA0008C809D80AE80BF8020E030E0A901C30102
:103AB000B2010E9465518823A1F1A5019401C701BB
:103AC000B6010E94F8500E94DC519B0177FF04C0B0
:103AD00022273327261B370BB901330F880B990B8D
:103AE0000E9414529B01AC01C301B2010E946551B6
:103AF00087FF17C0CC82DD82EE82FF826C817D81E0
:103B00008E819F81DF91CF91FF90EF90DF90CF90DA
:103B1000BF90AF909F908F907F906F905F904F90ED
:103B20000895488059806A807B80A301920160E0FB
:103B300070E080E89FE30E94F850A50194010E9484
:103B400021534B015C01A7019601C301B2010E9400
:103B500021539B01AC01C501B4010E94F9506C8353
:103B60007D838E839F83CACF8550883070F4E82F81
:103B7000F0E0E354F24E0C945955D01DD81DE01DD1
:103B8000E81DF01DF81D001E081E60937E2870932E
:103B90007F2868EB7EE184E00E94310481E0089593
:103BA000609380287093812862EB7EE185E0F4CFFA
:103BB00060938228709383286CEA7EE186E0ECCFE4
:103BC000609384287093852866EA7EE187E0E4CFDD
:103BD000609386287093872860EA7EE188E0DCCFD6
:103BE00060938828709389286AE97EE189E0D4CFC0
:103BF00060938A2870938B2864E97EE18AE0CCCFB9
:103C000060938C2870938D286EE87EE18BE0C4CFA2
:103C100060938E2870938F2868E87EE18CE0BCCF9B
:103C2000DC01ED91FD918081ED91FD919081ED910F
:103C3000FD916C9163708E2309F064609F2309F0FD
:103C40006860EDE2FEE1E60FF11D659565956D9307
:103C50006D917D918D919D91099423C01AC012C0E0
:103C600016C010C01EC009C014C013C006C019C0C1
:103C700009C00DC007C00DC014C062507040804024
:103C800090400BC0615070408040904006C06E5F15
:103C900001C06F5F7F4F8F4F9F4F9E938E937E9398
:103CA0006E9308958091A0289091A1280C94101EE5
:103CB00080919E2890919F280C94101E80919C28A2
:103CC00090919D280C94101E80919A2890919B2889
:103CD0000C94101E80919828909199280C94101E95
:103CE00080919628909197280C94101E809194288A
:103CF000909195280C94101E809192289091932871
:103D00000C94101E80919028909191280C94101E74
:103D100080918E2890918F280C94101E80918C2871
:103D200090918D280C94101E80918A2890918B2858
:103D30000C94101E80918828909189280C94101E54
:103D400080918628909187280C94101E8091842859
:103D5000909185280C94101E809182289091832840
:103D60000C94101E80918028909181280C94101E34
:103D700080917E2890917F280C94101E80917C2841
:103D800090917D280C94101E80917A2890917B2828
:103D90000C94101E80917828909179280C94101E14
:103DA00080917628909177280C94101ECF93DF9302
:103DB000EC018B85823060F4F894CE010E94101ED5
:103DC0006F81788589859A857894DF91CF91089560
:103DD000F894F6CF0F931F93CF93DF93EC01062F48
:103DE000142F70E060E0802F0E940B0761E070E00C
:103DF000802F0E94810770E060E0812F0E940B07F6
:103E000061E070E0812F0E948107802F90E0FC012B
:103E1000E65EF041A081A63008F04EC020E2A29FED
:103E2000D0011124BC5F9D01285F3F4F2883398357
:103E300080509141FC0140814C83812F90E0FC0136
:103E4000E65EF041E08170E060E0E63030F420E2D0
:103E5000E29FF0011124BF017C5F9B01285F3F4F6F
:103E60002A833B8380509141FC0130813D831F8236
:103E7000188619861A868BE39FE10197F1F7189649
:103E80002C91242381E009F480E0FB0190859323A9
:103E900009F082608E83BE01802F0E94B41D8B8743
:103EA000BE01812F0E94B41D9B85890F8B87DF91F6
:103EB000CF911F910F910895B0E0A0E0B4CF8F9201
:103EC0009F92AF92BF920F931F93CF93DF93CDB783
:103ED000DEB7A197CDBFDEBF19A2423008F44AE099
:103EE0008E010F5D1F4F842E912CB12CA12CA501AA
:103EF00094010E94C750E62FB901CA01EA302CF59F
:103F0000E05DD801EE938D01232B242B252B79F72F
:103F100090E080E0109769F0FD0101900020E9F742
:103F20003197AF014A1B5B0BBD018BEB9DE20E94F9
:103F30004506A196CDBFDEBFDF91CF911F910F91B6
:103F4000BF90AF909F908F900895E95CDACFCF92A9
:103F5000DF92EF92FF92CF93DF936B017C016DE2D2
:103F60008BEB9DE20E941B17EC0166277727CB01A4
:103F70006C197D098E099F094AE00E945F1F8C0F12
:103F80009D1FDF91CF91FF90EF90DF90CF9008952C
:103F9000009769F0FC0101900020E9F73197AF012B
:103FA000481B590BBC018BEB9DE20C94450690E03D
:103FB00080E0089540EA50E062E070E090E080E048
:103FC0000E94151B0E94A4088091E72A9091E82A7C
:103FD0008093E52A9093E62A863091059CF486E743
:103FE0009FEE0E94C81F8091E52A9091E62A8630B4
:103FF000910510F5880F991FFC01EE58F141808161
:10400000918115C089309105A9F740EA50E062E03E
:1040100070E090E080E00E94151B8BE79FEE0E940D
:10402000C81F8091E42A811104C080EE9FEE0C9499
:10403000C81F82E79FEEFBCF08958F929F92AF92A9
:10404000BF92CF92DF92EF92FF920F931F93CF9385
:10405000DF937C016B018A012417350710F030E0F3
:1040600020E0E901219740EF50E063E070E08AE052
:1040700090E00E94151BC7010E94C81F99E1E92E1C
:104080009CEFF92E8091682A9091692A0E94D61E91
:104090004B01940121703327232B11F594012E1924
:1040A0003F0912161306DCF16E157F05C9F08FEF7C
:1040B0009FEFC80FD91FD7FF35C0C00FD11F44E6EF
:1040C00050E063E070E080EA90E00E94151BFE0182
:1040D000EE0FFF1FEC0DFD1D808191810E94C81F16
:1040E00080916C2A90916D2A0E94AB09E0916C2A14
:1040F000F0916D2A808580FD10C082FF0EC0CE0138
:10410000DF91CF911F910F91FF90EF90DF90CF90B3
:10411000BF90AF909F908F9008957401B3CF81E0CE
:1041200090E0C7CFC017D10754F2C01BD10BC7CF47
:10413000CF92DF92EF92FF922091B92A211156C0BF
:1041400041110EC0C090A628D090A728E090A828C2
:10415000F090A928C616D706E806F90609F446C065
:104160006B017C01C092A628D092A728E092A828D3
:10417000F092A9284CE350E064E070E08CE390E01A
:104180000E94151B8091452890914628892B79F033
:1041900081EBC81684E0D806E104F10444F086E817
:1041A0009FEEFF90EF90DF90CF900C94C81FF7FE2A
:1041B00017C0C701B6010E94A71F20E030E040E809
:1041C0005FE360913128709132288091332890917B
:1041D00034280E946551882349F088E89FEEE1CF9A
:1041E0004AE0C701B6010E945F1FE7CFFF90EF9042
:1041F000DF90CF900895BC01990F880B990B97FD24
:104200000C94A71F4AE00C945F1FCF93DF93873F66
:104210002FEF920724F4DF91CF910C94FB20EC0157
:1042200097FF06C08DE89FEE0E94C81FCE01F3CF16
:104230008AE89FEECA30D105BCF78CE89FEE209744
:1042400099F78FE89FEEDF91CF910C94C81F7F9272
:104250008F929F92AF92BF92CF92DF92EF92FF9296
:104260000F931F93CF93DF93062F5A01882361F09A
:1042700040EA50E061E070E090E080E00E94151BB1
:1042800083E99FEE0E94C81F21E8C22E2AE2D22EA7
:10429000D0E0C0E010E03AE2732E011169C0AC1624
:1042A000BD0609F469C080910228909103288C17FB
:1042B0009D0729F5EE24EA94FE2CF601808091807A
:1042C00063E070E0C430D10514F462E070E04AE2CB
:1042D00050E0CE01837099279C01729EC001739EAD
:1042E000900D11240E94151BE092CD2DF092CE2D41
:1042F000E092CB2DF092CC2DC4010E94052111112A
:1043000007C011E0F60180819181892B09F410E04A
:104310002196F2E0CF0ED11CC830D10509F0BDCFF7
:104320008FEF9FEF8093CD2D9093CE2D8093CB2D4B
:104330009093CC2D112341F08091452890914628EF
:1043400011E0892B09F410E01093E32AA0920228CF
:10435000B0920328DF91CF911F910F91FF90EF90C2
:10436000DF90CF90BF90AF909F908F907F900895F7
:10437000AC16BD0609F09ECF87EEE82E89EFF82E29
:104380009CCF8F929F92AF92BF92CF92DF92EF928B
:10439000FF920F931F93CF93DF93962E7A0188237A
:1043A00061F040EA50E061E070E090E080E00E945F
:1043B000151B80EA9FEE0E94C81F81E2C82E88E28A
:1043C000D82ED0E0C0E09AE2892E911051C0EC16B0
:1043D000FD0609F451C080910428909105288C179E
:1043E0009D0721F50FEF1FEFF601A080B18063E07C
:1043F00070E0C430D10514F462E070E04AE250E0AD
:10440000CE01837099279C01829EC001839E900DEE
:1044100011240E94151B0093CD2D1093CE2D0093D7
:10442000CB2D1093CC2DC5010E940521219632E0A1
:10443000C30ED11CC830D10541F68FEF9FEF80939A
:10444000CD2D9093CE2D8093CB2D9093CC2DE092BB
:104450000428F0920528DF91CF911F910F91FF90D2
:10446000EF90DF90CF90BF90AF909F908F90089586
:10447000EC16FD0609F0B6CF07EE19EFB5CFEF92B7
:10448000FF920F931F93CF93DF930097A9F0409172
:104490004728509148286091492870914A284D3DFD
:1044A00055406105710544F02091002830910128A4
:1044B0002F3F3F4F09F450C02091D42D3091D52D7E
:1044C000232B51F42091C92D3091CA2D2A5F3F4FE3
:1044D0002093C92D3093CA2D2FED32E02093D42D97
:1044E0003093D52D1816190624F5EC018091472834
:1044F00090914828A0914928B0914A288D3D954037
:10450000A105B10584F1E0901329F09014290FE37F
:1045100010E028E330E048E350E066EB70E08BEB1E
:104520009DE20E9433128FEF9FEF809300289093BB
:1045300001288091D42D9091D52D892B49F080911F
:10454000C92D9091CA2D06978093C92D9093CA2D9D
:104550001092D42D1092D52DDF91CF911F910F91F4
:10456000FF90EF90089580910028909101288C177A
:104570009D07F9F2E0901A29F0901B290FE310E053
:1045800028E330E048E350E066EB70E08BEB9DE21F
:104590000E9433128CEB90E08093C72D9093C82D2E
:1045A0008EE690E08093C92D9093CA2DCE010E9493
:1045B000FB20C0930028D0930128BBCFFF920F931C
:1045C0001F93CF93DF93F62E2091402830914128FE
:1045D000AC01421B530B2817390714F59A0180933D
:1045E000402890934128E90121978091AF2A8823A0
:1045F00029F070E060E080E10E943A0710E000E0FE
:1046000061E070E080E10C171D0774F40E943A0726
:1046100070E060E080E10E943A070F5F1F4FF0CF2B
:104620009A01285F3F4FDBCF0E943A070E9445085E
:104630006093AB2A7093AC2A8093AD2A9093AE2AF4
:10464000C1E0C093AF2AFF2031F061E085E00E9415
:10465000EF04C093B02A80914028909141280196A0
:10466000DF91CF911F910F91FF900C943F22CF9338
:10467000DF93EC014CE050E061E070E080EC90E012
:104680000E94151B1C161D062CF4CE01DF91CF9144
:104690000C94FB20DF91CF9108951F93CF93DF936C
:1046A000182F8091C02AC6E0D0E081110AC0809105
:1046B000B12AC0913C28D0913D28882311F0C7E051
:1046C000D0E08FEF9FEF8093CD2D9093CE2D8093F0
:1046D000CB2D9093CC2D82E08093CF2D8093D02D45
:1046E00040EA50E0C930D10509F05DC062E070E0F9
:1046F00090E080E00E94151B8BE79FEE0E94C81F90
:104700008091E42A81114CC080EE9FEE0E94C81F68
:1047100084EB90E08093C72D9093C82DCEE1D0E03C
:10472000C093C92DD093CA2D8BEA9FEE0E94C81F5B
:104730008CEC90E08093C72D9093C82DC093C92D29
:10474000D093CA2D8DEA9FEE0E94C81F80913E280B
:1047500090913F280E9437231123D9F040EA50E07E
:1047600063E070E090E080E00E94151B8FEA9FEE0E
:104770000E94C81F49E150E063E070E084E890E0E7
:104780000E94151B8091952A9091962A01960E946D
:10479000FB2090E080E0DF91CF911F910C943F22AD
:1047A00082E79FEEB3CF61E070E090E080E00E948E
:1047B000151BCC0FDD1FCE58D14188819981A6CF22
:1047C0008091E42C9091E52C0297029750F480910F
:1047D00060288823C9F150E040E061E081E00E9458
:1047E00027218091D12C9091D22C0297029750F4DE
:1047F00080916128882389F150E040E061E081E008
:104800000E94C12180916228882329F081E00E94C2
:104810004D230E94DA1F10925C2810925D2810929E
:104820005E2810925F2810926028109261288FEF06
:104830009FEF8093632890936428809365289093DA
:104840006628109262280895409165285091662844
:1048500057FDC7CF61E080E0C2CF409163285091FF
:10486000642857FDCFCF61E080E0CACFCF92DF92BE
:10487000EF92FF920F931F93CF93DF93EC01088188
:1048800019816A817B81601B710B072E000C880BDC
:10489000990B0E9414529B01AC0160E070E080EC27
:1048A00091E40E946A516B017C0168857985601BE7
:1048B000710B072E000C880B990B0E9414529B0160
:1048C000AC01C701B6010E9421530E94DE530E9431
:1048D000DC51CB0197FF02C00C96FCCF6CE070E07E
:1048E0000E944555FC01EE0FFF1FEA5FF1418081F8
:1048F00091810197DF91CF911F910F91FF90EF90E0
:10490000DF90CF9008954F925F926F927F928F9237
:104910009F92AF92BF92CF92DF92EF92FF920F934E
:104920001F93CF93DF93CDB7DEB72E97CDBFDEBFFA
:10493000C0903128D0903228E0903328F09034286D
:10494000BC0104970CF0B2C06F5F7F4F072E000CC4
:10495000880B990B0E9414529B01AC0160E070E03F
:1049600080E89FE30E946A516093AA287093AB2865
:104970008093AC289093AD2820914528309146280B
:104980002230310561F421E02983A70196010E94BC
:104990006551811101C0198239813093AE28809010
:1049A000AA289090AB28A090AC28B090AD2841E008
:1049B0004983A7019601C501B4010E946551811187
:1049C00001C01982598150936A2AA7019601C50135
:1049D000B4010E946551882309F466C18091AE2814
:1049E000811162C18092312890923228A09233289E
:1049F000B092342860910A2870E090E080E00E9434
:104A00001452A50194010E9421530E94DC51AB0174
:104A10008091112990911229BA010E9445558093E5
:104A200011299093122980930B2990930C2960915E
:104A30004728709148288091492890914A280E94DF
:104A4000145269837A838B839C839B01AC0160EC55
:104A500071EE84E69CE40E946A51A50194010E94D3
:104A6000215320E030E044EB52E40E946A510E945E
:104A7000DE530E94E3516B017C010091442C1091A4
:104A8000452CD8018C918E7F8C938C9186708230CE
:104A900009F470C08430D9F0811120C044E0CC0CFE
:104AA000DD1CEE1CFF1C4A95D1F718C0635071093C
:104AB000072E000C880B990B0E9414526093AA28B1
:104AC0007093AB288093AC289093AD2868CF62E0B8
:104AD000F694E794D794C7946A95D1F780E090E074
:104AE000A1E0B0E08093522C9093532CA093542CCF
:104AF000B093552C9701442755272B873C874D872A
:104B00005E872093462C3093472C4093482C50933B
:104B1000492CC701B6018827992760934A2C7093C6
:104B20004B2C80934C2C90934D2C232B242B252BFA
:104B300009F444C0412C512C32016394A301920129
:104B400021503109410951092D833E834F835887F4
:104B50006130710581059105A9F4C701B6010E9474
:104B6000C7502B873C874D875E874D805E806F8066
:104B70007884E4CF53E0CC0CDD1CEE1CFF1C5A956E
:104B8000D1F7ACCF60934A2C70934B2C80934C2C74
:104B900090934D2C4092522C5092532C6092542C56
:104BA0007092552C2B853C854D855E852093462C37
:104BB0003093472C4093482C5093492C8091522C91
:104BC0009091532CA091542CB091552C0197A10990
:104BD000B1098093522C9093532CA093542CB093F2
:104BE000552C40914A2C50914B2C60914C2C70913B
:104BF0004D2C411551056105710561F04150510978
:104C00006109710940934A2C50934B2C60934C2CB2
:104C100070934D2C4091462C5091472C6091482C1C
:104C20007091492C40934E2C50934F2C6093502CF4
:104C30007093512C452B462B472B21F480914A2C05
:104C400090914B2CD8011C968D939C931D971A968E
:104C50001D921C921B978C9181608C9380914528AA
:104C600090914628892B01F5A501940169817A81EB
:104C70008B819C810E946A510E94DC5140E02E96FB
:104C8000CDBFDEBFDF91CF911F910F91FF90EF90CD
:104C9000DF90CF90BF90AF909F908F907F906F905C
:104CA0005F904F900C9498202E96CDBFDEBFDF9181
:104CB000CF911F910F91FF90EF90DF90CF90BF9019
:104CC000AF909F908F907F906F905F904F900895DE
:104CD0000F931F93CF93DF938091E72A9091E82A57
:104CE00088309105A9F440EA50E061E070E090E07E
:104CF00080E00E94151B8AEB9FEE0E94C81F109255
:104D0000402810924128DF91CF911F910F91089573
:104D10001092B12A1092C02A863091050CF04DC035
:104D20008091E52A9091E62A80933C2890933D2833
:104D300082309105D1F481E08093422880E00E9486
:104D40004D238091B12A811104C08091C02A88230B
:104D5000D1F240EA50E062E070E090E080E0DF9164
:104D6000CF911F910F910C94151B049739F70CE309
:104D700018E2C8E0D0E00E94804FBE010E94455575
:104D8000D8015E962D913C915F97FC01EE0FFF1FBD
:104D9000E45BF74D808191815E968D939C935F9744
:104DA000332720833183219702501109209719F767
:104DB0001092432810924428C1CF21E087309105FA
:104DC00009F020E02093B12A21E08630910509F016
:104DD00020E02093C02A099709F0B0CF8091E42AFF
:104DE00091E089278093E42A40EA50E062E070E095
:104DF00090E080E00E94151B8BE79FEE0E94C81F89
:104E00008091E42A81111AC080EE9FEE0E94C81F93
:104E10008091452890914628892B61F08091E42A61
:104E2000882349F0209145283091462881E021309F
:104E3000310509F080E08093E32A80CF82E79FEE7E
:104E4000E5CF20914528309146282230310509F0E0
:104E50004BC02091552A3091562A1216130624F47D
:104E60008217130609F040C0842F90E024E0959546
:104E700087952A95E1F78770613161F0623129F1F8
:104E8000603191F590E0019680933E2890933F2801
:104E90000C943723863040F590E02091E72A30913A
:104EA000E82A8217930701F18093E72A9093E82A72
:104EB0008093E52A9093E62A80916A2A882319F044
:104EC00010926A2A08950C946826873069F0282F7A
:104ED00030E0843020F0C90103970C94832487E0EC
:104EE00090E0821B930BF9CF0895CF93DF938091CD
:104EF0003C2890913D2882309105E1F150F4C09119
:104F00003E28D0913F2821970197C1F0D0E0C0E022
:104F100015C0C0914C28D0914D288430910571F076
:104F20000597A1F70E94804F892F990F990B6091E7
:104F30003E2870913F280E944555EC01109243286D
:104F40001092442860E0CE010E94DE228091D12C94
:104F50009091D22C0197029788F4CC0FDD1FCF5D82
:104F6000D74D888199818093A92A9093AA2ADF91AD
:104F7000CF91089581E080934228C8CF81E090E0EE
:104F8000F2CF0F931F93CF93DF938091E42A88236E
:104F9000A9F088E790E0809316289093172881E085
:104FA0008093572A80914B288823B1F181E0809328
:104FB000B22ADF91CF911F910F9108958091E42C37
:104FC0009091E52C0197029768F7C0914028D09105
:104FD0004128CE01029608E010E0B8010E94455534
:104FE000FC01EE0FFF1FEF57F54D20813181265A4E
:104FF0003F4FCE010196B8010E944555FC01EE0FCE
:10500000FF1FEF57F54D80819181281B390B2093AD
:10501000162830931728C6CFDF91CF911F910F919B
:105020000C9475278091E32A811122C08091452834
:1050300090914628019721F48091D12A81110AC0CC
:105040008091452890914628029771F48091D22A48
:10505000882351F08091B22A882359F01092B22A05
:105060000E9475271092B32A1092D12A1092D22A48
:10507000089581E08093B32AF7CF0E94BC56CF9267
:10508000DF92EF92FF920F93FC01C12CB9E0DB2E6F
:10509000BDE3EB2EF12CC082D182E282F382148236
:1050A000158281E090E086839783C0901128D0908C
:1050B0001228E0901328F0901428F694E794D794DF
:1050C000C79490E04C155D056E057F0540F4F6949D
:1050D000E794D794C7949F5F9630A1F797E0046058
:1050E0000187892F8095A82FA170B0E084E0AA0FD6
:1050F000BB1F8A95E1F791629A2B80E0232B09F47C
:1051000080E4982B90870F91FF90EF90DF90CF90E5
:1051100008950F931F93CF93DF93CDB7DEB72A97F0
:10512000CDBFDEBF8C01FC01878181110CC01086D0
:105130001186128613861486158616861786108A9F
:10514000118A81E087838091E305F8019681892B9C
:105150008093E30561E070E083810E940B0761E0CA
:1051600070E0F80184810E940B078091C10884607F
:105170008093C1088091C00881628093C0084091EB
:105180005C2C50915D2C60915E2C70915F2C009195
:10519000602C2091622C3091632CCE0101960E94EC
:1051A0003F2899858A859093C0088093C1082A96E4
:1051B000CDBFDEBFDF91CF911F910F910895CF92A8
:1051C000DF92EF92FF920F931F93CF93DF93EC0147
:1051D0006A017B01C114D104E104F10439F4C12C4A
:1051E00088E4D82E88EEE82EFF24F394FE01FF9683
:1051F000C082D182E282F38281E28DAF80E28EAF03
:10520000369610818FA987FD09C061E070E00E9489
:105210000B0761E070E08FA90E94810761E070E0F8
:1052200088AD0E940B0761E070E088AD0E948107A5
:105230008DA981114DC0C9A2DAA2EBA2FCA2812FD7
:1052400090E08DA39EA381E090E08FA398A7812F8B
:1052500090E0B0E0A0E089A79AA7ABA7BCA78F8D8C
:1052600098A184569C4221F484E69CE20E948928FD
:105270008EA987FD86C061E070E00E940B0761E0A7
:1052800070E08EA90E94810764E670E080E090E003
:105290000E94740870E060E08EA90E94810764E6B5
:1052A00070E080E090E00E94740861E070E08EA9F8
:1052B0000E94810768EC70E080E090E0DF91CF9180
:1052C0001F910F91FF90EF90DF90CF900C94740896
:1052D0000AE11FEEF12C8130E1F461E070E08AA573
:1052E0000E940B0770E060E08AA50E94810761E0E0
:1052F00070E08CA50E940B0770E060E08CA50E9416
:1053000081078BA587FDB4CF70E060E00E940B079A
:10531000AFCFF80181918F01863080F5F0E28F9F49
:10532000C00111249C5F04962F8D38A128173907DE
:1053300051F461E070E08F2D0E940B0770E060E097
:105340008F2D0E948107F39426E1F212E2CF61E0F3
:1053500070E08EA50E940B0761E070E08EA50E94B0
:1053600081078FA587FD84CF61E070E00E940B0765
:1053700061E070E08FA50E9481077ACF90E080E025
:10538000D2CFDF91CF911F910F91FF90EF90DF90DF
:10539000CF9008955F926F927F928F929F92AF927B
:1053A000BF92CF92DF92EF92FF920F931F93CF9312
:1053B000DF93CDB7DEB76297CDBFDEBF3C010B8771
:1053C0001C872D873E87042F4F87588B698B7A8BDC
:1053D00029893A894B855C856D857E85CE0101964C
:1053E0000E943F2859841A85D30118968C918823EE
:1053F00019F081FF18C0F8945092C0081093C108AA
:105400006296CDBFDEBFDF91CF911F910F91FF90CC
:10541000EF90DF90CF90BF90AF909F908F907F9054
:105420006F905F90089580FFE7CFF30182849384AB
:10543000A484B584C12CD12C7601B0E09401A501DF
:10544000B601C701A0E00E948B55A9F1217030E0A0
:1054500040E050E060E070E080E090E00E948B551A
:10546000E9F090E080E0B03370F48B2F869586955C
:105470008695F0E28F9FC0011124805F9B4F2B2FF8
:105480002770820F911DFC01408193012B0F311D6C
:10549000F901428BFC012081287F20839401A50122
:1054A000B601C70101E00E94705549015A016B0124
:1054B0007C01BF5FC3CFD3011E968D909D90AD90B0
:1054C000BC905197C12CD12C7601B0E29401A5017A
:1054D000B601C701A0E00E948B5509F48DCF217061
:1054E00030E040E050E060E070E080E090E00E945A
:1054F0008B55E9F090E080E0B03370F48B2F869507
:1055000086958695E0E28E9FC0011124805F9B4FB7
:105510002B2F2770820F911DFC01408193012B0FCF
:10552000311DF901428BFC012081287F20839401E9
:10553000A501B601C70101E00E94705549015A0159
:105540006B017C01BF5FC2CF0C943356FF920F9367
:105550001F93CF93DF938C01EB01F8800E943450AE
:10556000F81621F06F2DC8010E943C50CE01DF914A
:10557000CF911F910F91FF9008950F931F93CF9399
:10558000DF938C01EB010E9434508883C80101969F
:105590000E9434508983CE01DF91CF911F910F91EA
:1055A0000895FF920F931F93CF93DF93EC018B012C
:1055B000FB01F0800E943450F81621F06F2DCE01CF
:1055C0000E943C50F801F1802196CE010E94345097
:1055D000F81621F06F2DCE010E943C50C801DF91DA
:1055E000CF911F910F91FF900895CF93DF93C0E16A
:1055F000D0E0BE016F5E774DCE010E94D12A229687
:10560000C032D105B1F7DF91CF910895CF93DF93E9
:10561000C4E2D0E0BE01635A754DCE010E94D12A8A
:105620002296C433D105B1F7DF91CF910895CF937E
:10563000C62F80934B282AE530E02093162830931C
:10564000172861E0682784E00E94EF0460914B28EE
:1056500086E00E94EF04CC2391F00E94C127809144
:10566000912A81110E94062B8091922A81110E9419
:10567000F52A1092922A1092912ACF910895809142
:10568000E42A882361F388E790E0809316289093BA
:1056900017281092572AE3CF8091452890914628E9
:1056A000029721F460E080E00C94172B089580911C
:1056B000452890914628029771F40E943F1B8FEF76
:1056C0009FEF809311299093122960E081E00E945E
:1056D000172B0C945C1B08958091452890914628C7
:1056E000029791F40E943F1B8FEF9FEF8093112947
:1056F0009093122980930B2990930C2961E081E00B
:105700000E94172B0C945C1B089590E00C9434506D
:10571000882349F086E00E94852B91E0811101C029
:1057200090E090931529809115292FE130E088238E
:1057300011F020E038EF20931A2930931B2920EE36
:105740003FEF882311F02FEF3FEF2093182930937C
:105750001929811107C08AE090E080931329909362
:105760001429089580E090EAF8CF6F927F928F928B
:105770009F92AF92BF92CF92DF92EF92FF920F93E0
:105780001F93CF93DF93CDB7DEB7CA54D109CDBFF6
:10579000DEBFD82E81E00E94882B1092B92A70E0DB
:1057A00060E08BEB9DE20E94C4188091152861E0B7
:1057B000811163E08BEB9DE20E94B310E0901A2907
:1057C000F0901B290DE110E020EF30E050E040E0C8
:1057D00070E060E08BEB9DE20E9433128FEF9FEF51
:1057E0008093CD2D9093CE2D8093CB2D9093CC2D67
:1057F0008CE390E08093C72D9093C82D85E090E0D6
:105800008093C92D9093CA2D82E08093CF2D8093F1
:10581000D02D85EC9FEE0E94C81FDD2009F413C235
:105820008AE090E08093C72D9093C82D8EE190E0A0
:105830008093C92D9093CA2D80ED9FEE0E94C81FC2
:1058400068EE73E080E090E00E94740880E1E6E892
:10585000FDEEDE01D39601900D928A95E1F7FE01EF
:10586000B39680E1DF011D928A95E9F77E01B3E3EB
:10587000EB0EF11C8F013F01470140E1C42ED12CFA
:10588000BE016D5B7F4FC6010E94BD2A2596AEAC5E
:10589000BFAC2597D401AD92BD924D01BE016F5FA3
:1058A0007F4FC60144960E94BD2AB1E0AB1AB108F1
:1058B00049815A81E8E0AE16B10438F481E09A01DA
:1058C000245C3F4F2937310508F080E0D3014D9328
:1058D0005D933D0181115AC084E00E94852B91E0C7
:1058E000811101C090E09093372888E00E94852BB9
:1058F00090E08093552A9093562A8AE00E94852B47
:1059000091E0811101C090E09093742A8EE00E9492
:10591000852B90E0809316299093172980916E2A09
:1059200090916F2A0E94AB0980916C2A90916D2A08
:105930000E94AB09E0916C2AF0916D2A808580FD70
:10594000FEC140EF50E062E070E08AE090E00E942B
:10595000151B85ED9FEE0E94C81F80916E2A9091C5
:105960006F2ADC0118962C9120FF07C0E0916C2A69
:10597000F0916D2A208520FD29C00E94AB098091FD
:105980006C2A90916D2A0E94AB09E7CFE2E0CE0E1F
:10599000D11CF0E2CF16D10409F072CFA1E2B8E237
:1059A00041E85AE2C7014096F701219131917F0108
:1059B0002D933D93F801219131918F01FA012193AB
:1059C0003193AF018E159F0579F786CF809196EDC3
:1059D000909197EDA09198EDB09199ED2B968CAFA9
:1059E0009DAFAEAFBFAF2B972091372881E028271E
:1059F00030E042E050E0BE01695B7F4F83EE9FEEF6
:105A00000E941D2021E0892B09F020E020933728F7
:105A100067E378E284E090E00E94A62A80919AED04
:105A200090919BEDA0919CEDB0919DED27968CAF50
:105A30009DAFAEAFBFAF27972091152930E042E070
:105A400050E0BE016D5B7F4F80EF9FEE0E941D20F6
:105A500021E0019709F020E02093152965E179E222
:105A600086E090E00E94A62A2091742A81E02827EF
:105A700030E042E050E0BE01695B7F4F88EF9FEE6F
:105A80000E941D2021E0892B09F020E02093742A38
:105A900064E77AE28AE090E00E94A62A2091152825
:105AA00081E0282730E042E050E0BE01695B7F4F93
:105AB00084E090EF0E941D2021E0892B09F020E076
:105AC0002093152865E178E28CE090E00E94A62AF8
:105AD000209116293091172943E050E06BE078E2DD
:105AE00080E190EF0E941D20809316299093172942
:105AF00066E179E28EE090E00E94D12A8091162939
:105B00009091172963E070E00E944555FC01EE0F6B
:105B1000FF1FE050F241808180930A2882E2EEE983
:105B2000FDEEDE01119601900D928A95E1F720912C
:105B3000552A3091562A41E150E0BE016F5F7F4FF8
:105B400086E190EF0E941D208093552A9093562A5B
:105B500065E57AE288E090E00E94D12A80E00E9428
:105B6000B52BBE016D5B7F4F90E080E00E94BD2AA7
:105B700025968EAD9FAD25971816190624F48093AF
:105B8000082890930928BE016F5F7F4F82E090E064
:105B90000E94BD2A89819A811816190624F48093DF
:105BA00006289093072887E190E00E949755FC0112
:105BB0002091062830910728409108285091092803
:105BC0008FEF9FEF8387948785879687838B948B4E
:105BD00088E090E0858B968B4083518322833383CA
:105BE0001086118682E090E08483958384E190E0C2
:105BF00086839783E093BE2AF093BF2AE091722AAE
:105C0000F091732AF8941782108611861286789480
:105C1000E091682AF091692AF8941782108611861B
:105C20001286789487E090E08093662A9093672AA2
:105C30008091552A9091562A80939B2D90939C2D6C
:105C400080E00E94882B1092C72D1092C82D04E589
:105C500010E00093C92D1093CA2D8FE490EF0E949D
:105C6000C81F1092C72D1092C82D8FE690E0809328
:105C7000C92D9093CA2D8BE590EF0E94C81F80E03C
:105C80000E944D2380913E2890913F280E94372307
:105C900084E890E08093C72D9093C82D0093C92D80
:105CA0001093CA2D88E090E00E94FB208FEF9FEFB9
:105CB00080934528909346280E94B62FE0901A2999
:105CC000F0901B2903E410E02CE330E046E350E0C1
:105CD00064EB70E08BEB9DE20E943312E090182998
:105CE000F09019292CE330E046E350E064EB70E0DB
:105CF0008BEB9DE20E94ED17E0901829F090192996
:105D000001E410E02AE330E047E350E065EB70E0A7
:105D10008BEB9DE20E94ED17C65BDF4FCDBFDEBF70
:105D2000DF91CF911F910F91FF90EF90DF90CF9077
:105D3000BF90AF909F908F907F906F900895E0916B
:105D40006E2AF0916F2A808580FD0BCF40EF50E0E6
:105D500061E070E090E080E00E94151B8FE190EF21
:105D60000E94C81F80916E2A90916F2AFC012085A5
:105D700020FF07C0E0916C2AF0916D2A208520FD5C
:105D800009C00E94AB0980916C2A90916D2A0E94F3
:105D9000AB09E8CF1092C72D1092C82D89E3E82EE9
:105DA000F12CE092C92DF092CA2D89E290EF0E9469
:105DB000C81F60ED77E080E090E00E94740884E105
:105DC0000E9423080FEF13E09801281B390B25963A
:105DD0002EAF3FAF259798E7C92ED12CC092C72D83
:105DE000D092C82DE092C92DF092CA2D81E390EF98
:105DF0000E94C81F25968EAD9FAD25970E94FB205F
:105E000086E390EF0E94C81F68EE73E080E090E0A8
:105E10000E9474081092C72D1092C82D24E5E22E1E
:105E2000F12CE092C92DF092CA2D88E390EF0E94E8
:105E3000C81F60ED77E080E090E00E94740884E184
:105E40000E942308D801A81BB90BCD01A983BA83EE
:105E5000C092C72DD092C82DE092C92DF092CA2DC4
:105E60000E94FB2025968EAD9FAD25978D599F4FA3
:105E700029813A8182179307DCF084E10E9423088C
:105E8000F801E81BF90BE983FA8344E650E063E08C
:105E900070E088E790E00E94151B89819A810E943A
:105EA000FB2064E670E080E090E00E947408DACFA6
:105EB00088E790E08093C72D9093C82D8FE690E0FF
:105EC0008093C92D9093CA2D80E490EF0E94C81F43
:105ED0001092C72D1092C82D8AE890E08093C92DAA
:105EE0009093CA2D25968EAD9FAD2597843893400B
:105EF000C4F589819A81883E93409CF583E490EFB4
:105F00000E94C81F25968EAD9FAD259780930828C7
:105F10009093092889819A81809306289093072875
:105F200068E078E290E080E00E94D12A66E078E2C2
:105F300082E090E00E94D12A68EB7BE080E090E074
:105F40000E947408F12CE12C07E810E020EF30E00B
:105F50004CE150E070E060E08BEB9DE20E94331278
:105F600000CE88E490EF0E94C81FE6CFEF92FF9228
:105F70000F931F938FE00E942308893E23E092072E
:105F800074F4833523E092070CF077C085369105D1
:105F90000CF076C01F910F91FF90EF90089581E073
:105FA00090E020914528309146282817390791F331
:105FB000809345289093462860E087E00E94EF0494
:105FC00070E060E080E10E943A07F12CE12C0BE1E7
:105FD00010E028E730E04CE650E06CE370E08BEB3B
:105FE0009DE20E94331288E790E08093C72D909342
:105FF000C82D8FE690E08093C92D9093CA2D809193
:106000004528909146288130910509F45AC0D8F16D
:10601000029709F45BC00E943F1B80914528909134
:106020004628892B61F08091E42A882349F0209149
:1060300045283091462881E02130310509F080E083
:106040008093E32A80913728882309F4A3CF0E9404
:10605000A4086093BA2A7093BB2A8093BC2A9093B9
:10606000BD2A8091B92A882309F494CF80E01F913A
:106070000F91FF90EF900C94B52B82E090E091CFC0
:1060800090E080E08ECF8EE890EF0E94C81F609174
:106090004728709148288091492890914A280E9469
:1060A0001452209131283091322840913328509158
:1060B00034280E946A510E94DC5141E00E949820DD
:1060C000AACF83E990EF0E94C81FA5CF88E990EF7F
:1060D000FACF4F925F926F927F928F929F92AF9280
:1060E000BF92CF92DF92EF92FF920F931F93CF93C5
:1060F000DF93CDB7DEB72E97CDBFDEBF80914528A9
:1061000090914628019709F088C182E00E94FE071D
:1061100021E030E0892B11F030E020E02093D52AF7
:106120003093D62A82E00E94FE07019709F475C1D8
:106130002091E32A298381E082278093D12A0E943B
:1061400045084B015C013981332309F42EC180914C
:106150000D2990910E29A0910F29B0911029A50128
:106160009401281B390B4A0B5B0BCA01B9010E9431
:10617000125269837A838B839C8320E030E044EB66
:1061800052E40E946A5120E030E040E05FE30E9468
:10619000F9500E94DC516B01770FEE08FF08009167
:1061A000442C1091452CD8018C918E7F8C938C912E
:1061B0008670823009F45FC0843051F081110FC0C5
:1061C00044E0CC0CDD1CEE1CFF1C4A95D1F707C047
:1061D00062E0F694E794D794C7946A95D1F780E08B
:1061E00090E0A1E0B0E08093522C9093532CA093C8
:1061F000542CB093552C9701442755272B873C8767
:106200004D875E872093462C3093472C4093482C33
:106210005093492CC701B6018827992760934A2CCF
:1062200070934B2C80934C2C90934D2C232B242B30
:10623000252B09F444C0412C512C32016394A30155
:10624000920121503109410951092D833E834F8329
:1062500058876130710581059105A9F4C701B60120
:106260000E94C7502B873C874D875E874D805E809C
:106270006F807884E4CF53E0CC0CDD1CEE1CFF1C57
:106280005A95D1F7ACCF60934A2C70934B2C8093E6
:106290004C2C90934D2C4092522C5092532C609247
:1062A000542C7092552C2B853C854D855E85209312
:1062B000462C3093472C4093482C5093492C809186
:1062C000522C9091532CA091542CB091552C0197A5
:1062D000A109B1098093522C9093532CA093542C74
:1062E000B093552C40914A2C50914B2C60914C2CE2
:1062F00070914D2C411551056105710561F04150BA
:1063000051096109710940934A2C50934B2C6093B9
:106310004C2C70934D2C4091462C5091472C609101
:10632000482C7091492C40934E2C50934F2C6093E5
:10633000502C7093512C452B462B472B21F48091E8
:106340004A2C90914B2CD8011C968D939C931D97B1
:106350001A961D921C921B978C9181608C93C5019B
:10636000B4010E9412526B017C0120E030E040EC4D
:106370005FE369817A818B819C810E9421539B011B
:10638000AC01C701B6010E94F95020E030E04AE7B5
:1063900054E40E946A510E94E3516093DF2A709393
:1063A000E02A8093E12A9093E22A80920D2990922C
:1063B0000E29A0920F29B09210298091C02A811134
:1063C00004C08091D12A882341F180913728882305
:1063D00021F10E94A4086093BA2A7093BB2A80938B
:1063E000BC2A9093BD2A8091B92A8823B1F080E01D
:1063F0002E96CDBFDEBFDF91CF911F910F91FF9001
:10640000EF90DF90CF90BF90AF909F908F907F9054
:106410006F905F904F900C94B52B2E96CDBFDEBF42
:10642000DF91CF911F910F91FF90EF90DF90CF9070
:10643000BF90AF909F908F907F906F905F904F90A4
:1064400008950E94A4086093B52A7093B62A809399
:10645000B72A9093B82A8091972A9091982A63E05E
:1064600070E00E944555892B01F564EF71E080E0F2
:1064700090E00E94740870E060E08BEB9DE20E9467
:10648000C41864EF71E080E090E00E9474080E94FC
:10649000DC4F23E030E040E050E00E9464506E5F4B
:1064A0007F4F6093192870931A280E94DC4F23E0D5
:1064B00030E040E050E00E9464506093A72A70935F
:1064C000A82A0E94DC4F22E330E040E050E00E9426
:1064D0006450FB014091992A50919A2A4115510527
:1064E00009F47CC04330510509F478C02091C32DD4
:1064F0003091C42D261B370B20939B2A30939C2A66
:106500004230510534F0E091C52DF091C62DE61BC7
:10651000F70BE0939D2AF0939E2A2091C32D309192
:10652000C42D4230510514F430E020E02093A52A18
:106530003093A62A4115510529F030E020E0433080
:10654000510521F42091C52D3091C62D2093A12A0B
:106550003093A22A2091C32D3091C42D4230510591
:1065600014F030E020E02093A32A3093A42A4115B0
:10657000510539F04330510599F14091C52D5091A5
:10658000C62D40939F2A5093A02A0E94DC4F2DE7EE
:1065900030E040E050E00E946450675E7F4F8F4FD4
:1065A0009F4F0E94145220E030E048E452E40E94E1
:1065B0006A5160931D2870931E2880931F28909322
:1065C00020280E94DC4F2FEF3FEF40E050E00E9478
:1065D000645060931B2870931C2808959B018CCFF6
:1065E00050E040E0CECF3F924F925F926F927F9209
:1065F0008F929F92AF92BF92CF92DF92EF92FF92D3
:106600000F931F93CF93DF93CDB7DEB72A97CDBFFC
:10661000DEBF8091452890914628029709F0F6C286
:1066200080911129909112290196809311299093BC
:10663000122980910B2990910C29019680930B29A6
:1066400090930C292091092930910A292F5F3F4FFF
:1066500029873A872093092930930A290E944508FF
:106660006B017C0180900D2990900E29A0900F293C
:10667000B090102981149104A104B10409F4BDC0A3
:106680008C149D04AE04BF0408F0B7C040903828B5
:106690005090392860903A2870903B2860910A28E1
:1066A00070E090E080E00E941452209131283091F7
:1066B000322840913328509134280E9421539B0165
:1066C000AC0160E070E68AE697E40E946A51698353
:1066D0007A838B839C83C701B6010E9412526D831B
:1066E0007E838F839887C501B4010E9412529B015B
:1066F000AC016D817E818F8198850E94F8509B014D
:10670000AC0169817A818B819C810E946A5120E071
:1067100030E04AE754E40E9421534B015C01809130
:10672000072990910829FC01EE0FFF1FEE0FFF1FB4
:10673000E552F74D80829182A282B38201966BE08E
:1067400070E00E9445558093072990930829898518
:106750009A850B971CF18CE2EBEDF8E2AFEAB8E218
:1067600001900D928A95E1F725E03BE144E050E08D
:106770006BE070E08FEA98E20E94C74D8091C328D9
:106780009091C428A091C528B091C628809338283C
:1067900090933928A0933A28B0933B28A301920103
:1067A000609138287091392880913A2890913B283F
:1067B0000E94F8500E94DC519B0177FF04C0222701
:1067C0003327261B370BB901330F880B990B0E9417
:1067D0001452A30192010E946A5120E030E040E887
:1067E0005EE30E941C53181644F48092382890925D
:1067F0003928A0923A28B0923B28C0920D29D09215
:106800000E29E0920F29F0921029409038285090DC
:10681000392860903A2870903B28B301A2018EEB92
:106820009CE20E943B1D0E94DE5369837A838B8326
:106830009C8300910A2810E0B801012E000C880BFF
:10684000990B0E9414526B017C01209131283091E8
:10685000322840913328509134280E9421530E94BD
:10686000DE530E94DC516D837E832091E42A222333
:1068700019F13090572A072E000C880B990B0E94B3
:1068800014524B015C018D819E8163E070E00E9497
:106890004555072E000C880B990B0E9414529B0142
:1068A000AC01C501B401332009F49CC00E94F95029
:1068B0000E94DC516D837E83809111299091122971
:1068C000ED81FE818E179F0709F0B5C18091572A8F
:1068D00091E089278093572A10921129109212294A
:1068E0008091AE28882309F44BC180910B299091A7
:1068F0000C29B8010E944555892B09F041C110921D
:10690000AE2810920B2910920C298090AA28909002
:10691000AB28A090AC28B090AD28809231289092FE
:106920003228A0923328B092342880914528909143
:106930004628029709F059C0A7019601C301B20188
:106940000E94215320E030E040EC51E40E946A5163
:106950000E94DE530E94DC5140E00E94982060912A
:106960004728709148288091492890914A280E9490
:1069700014529B01AC0160EC71EE84E69CE40E9431
:106980006A5120913128309132284091332850911A
:1069900034280E94215320E030E044EB52E40E946E
:1069A0006A510E94DE530E94E3516B017C012091E9
:1069B000442C3091452C2D833E83F90180818E7FBC
:1069C000808380818670823009F46DC0843019F133
:1069D000811128C0A4E0CC0CDD1CEE1CFF1CAA9584
:1069E000D1F720C00E94F85063CF80914528909144
:1069F0004628892B09F0B3CF609147287091482829
:106A00008091492890914A280E941452A50194012E
:106A10000E946A519FCF12E0F694E794D794C794EE
:106A20001A95D1F780E090E0A1E0B0E08093522C7D
:106A30009093532CA093542CB093552C970144273A
:106A400055272093462C3093472C4093482C509345
:106A5000492CC701B6018827992760934A2C709367
:106A60004B2C80934C2C90934D2C211531054105D6
:106A70005105C9F1412C512C32016394530142015B
:106A8000F1E08F1A9108A108B10861307105810504
:106A9000910589F4C701B601A50194010E94C75070
:106AA00024013501EBCFB3E0CC0CDD1CEE1CFF1C48
:106AB000BA95D1F7B7CF60934A2C70934B2C809343
:106AC0004C2C90934D2C4092522C5092532C60920F
:106AD000542C7092552C2093462C3093472C409385
:106AE000482C5093492C8091522C9091532CA0917A
:106AF000542CB091552C0197A109B1098093522CC7
:106B00009093532CA093542CB093552C40914A2C25
:106B100050914B2C60914C2C70914D2C411551058E
:106B20006105710561F04150510961097109409396
:106B30004A2C50934B2C60934C2C70934D2C4091CD
:106B4000462C5091472C6091482C7091492C4093D1
:106B50004E2C50934F2C6093502C7093512C452BFE
:106B6000462B472B21F480914A2C90914B2CED81A0
:106B7000FE81848795871286138680818160808359
:106B800080910D2990910E29A0910F29B091102983
:106B9000892B8A2B8B2B79F169817A818B819C815E
:106BA0000E94DC516B017C018091CF2A9091D02A08
:106BB000092E000CAA0BBB0BC816D906EA06FB0669
:106BC000D1F0A0910A28B0E0A70196010E9483505D
:106BD00028E130E040E050E00E946450CA01B90171
:106BE0000E9414520E94DC5140E00E949820C09202
:106BF000CF2AD092D02A80914B2881110E945C1B11
:106C000081E090E08093D52A9093D62A2A96CDBF32
:106C1000DEBFDF91CF911F910F91FF90EF90DF903A
:106C2000CF90BF90AF909F908F907F906F905F902C
:106C30004F903F9008952D813E8137FF04C02F5F14
:106C40003F4F2D833E83ED81FE81F595E795E81753
:106C5000F907E4F61092D52A1092D62AD7CF1F92C0
:106C60000F920FB60F9211242F933F934F935F9380
:106C70006F937F938F939F93AF93BF93EF93FF9304
:106C800085E00E947206FF91EF91BF91AF919F91B5
:106C90008F917F916F915F914F913F912F910F90C5
:106CA0000FBE0F901F9018951F920F920FB60F9264
:106CB00011242F933F934F935F936F937F938F9301
:106CC0009F93AF93BF93EF93FF9384E00E9472066C
:106CD000FF91EF91BF91AF919F918F917F916F91B4
:106CE0005F914F913F912F910F900FBE0F901F908A
:106CF00018951F920F920FB60F9211242F933F9366
:106D00004F935F936F937F938F939F93AF93BF93B3
:106D1000EF93FF9383E00E947206FF91EF91BF9182
:106D2000AF919F918F917F916F915F914F913F9123
:106D30002F910F900FBE0F901F9018951F920F92DA
:106D40000FB60F9211242F933F934F935F936F933E
:106D50007F938F939F93AF93BF93EF93FF9382E0C3
:106D60000E947206FF91EF91BF91AF919F918F9119
:106D70007F916F915F914F913F912F910F900FBE37
:106D80000F901F9018951F920F920FB60F9211241B
:106D90002F933F934F935F936F937F938F939F9323
:106DA000AF93BF93EF93FF9381E00E947206FF9130
:106DB000EF91BF91AF919F918F917F916F915F9173
:106DC0004F913F912F910F900FBE0F901F901895EC
:106DD0001F920F920FB60F9211242F933F934F9350
:106DE0005F936F937F938F939F93AF93BF93EF9333
:106DF000FF9380E00E947206FF91EF91BF91AF91E7
:106E00009F918F917F916F915F914F913F912F91C2
:106E10000F900FBE0F901F9018951F920F920FB6F4
:106E20000F9211242F933F934F935F936F937F9310
:106E30008F939F93AF93BF93EF93FF9384EF9CE265
:106E40000E948D05FF91EF91BF91AF919F918F911E
:106E50007F916F915F914F913F912F910F900FBE56
:106E60000F901F9018951F920F920FB60F9211243A
:106E70002F933F934F935F936F937F938F939F9342
:106E8000AF93BF93EF93FF9384EF9CE20E94AB0616
:106E9000FF91EF91BF91AF919F918F917F916F91F2
:106EA0005F914F913F912F910F900FBE0F901F90C8
:106EB00018951F920F920FB60F9211242F933F93A4
:106EC0004F935F936F937F938F939F93AF93BF93F2
:106ED000EF93FF9389EA9BE20E948D05FF91EF916A
:106EE000BF91AF919F918F917F916F915F914F91E2
:106EF0003F912F910F900FBE0F901F9018951F92EA
:106F00000F920FB60F9211242F933F934F935F93DD
:106F10006F937F938F939F93AF93BF93EF93FF9361
:106F200089EA9BE20E94AB06FF91EF91BF91AF917E
:106F30009F918F917F916F915F914F913F912F9191
:106F40000F900FBE0F901F9018951F920F920FB6C3
:106F50000F9211242F933F934F935F936F937F93DF
:106F60008F939F93AF93BF934091452A5091462AA8
:106F70006091472A7091482A8091432A9091442A2F
:106F800020914F2A3091502A420F531F611D711DCD
:106F900020914D2A30914E2A820F931F883E23E084
:106FA000920730F0885E93404F5F5F4F6F4F7F4F87
:106FB0008093432A9093442A4093452A5093462A2B
:106FC0006093472A7093482A8091492A90914A2ACF
:106FD000A0914B2AB0914C2A0196A11DB11D80931E
:106FE000492A90934A2AA0934B2AB0934C2A81E0D5
:106FF0008093B60ABF91AF919F918F917F916F91CE
:107000005F914F913F912F910F900FBE0F901F9066
:1070100018951F920F920FB60F9211242F933F9342
:107020004F935F936F937F938F939F93AF93BF9390
:10703000EF93FF9380914E2C90914F2CA091502C68
:10704000B091512C0197A109B10980934E2C9093D6
:107050004F2CA093502CB093512C181619061A06D9
:107060001B063CF1892B8A2B8B2BB9F18091462C86
:107070009091472CA091482CB091492C0097A105E4
:10708000B10591F080934E2C90934F2CA093502CEF
:10709000B093512CE091442CF091452C8091522CCE
:1070A0009091532C84879587E091562CF091572C22
:1070B000099581E08093A60AFF91EF91BF91AF916E
:1070C0009F918F917F916F915F914F913F912F9100
:1070D0000F900FBE0F901F90189540914A2C509121
:1070E0004B2C60914C2C70914D2C41155105610534
:1070F0007105A9F0E091442CF091452C4487558707
:1071000082859385B0E0A0E084179507A607B707AE
:1071100084F28091522C9091532C84879587809192
:10712000462C9091472CA091482CB091492C8093EB
:107130004E2C90934F2CA093502CB093512CB4CF45
:107140001F920F920FB60F9211242F933F934F93DC
:107150005F936F937F938F939F93AF93BF93CF93DF
:10716000EF93FF93C091AB08C2FF0AC01092362A7A
:107170001092352A1092342A84E00E94450C14C0E3
:10718000C6FF2FC08091332A813051F48091362A76
:10719000E091312AF091322A90E009951092332A39
:1071A000C0FF14C00E94550CFF91EF91CF91BF9189
:1071B000AF919F918F917F916F915F914F913F918F
:1071C0002F910F900FBE0F901F90189580E4809321
:1071D000AB0881E00E94450C8091AB0885FFE4CFAD
:1071E000E1CFC7FF5CC0C3FF08C01092362A1092DF
:1071F000352A1092342A83E0C0CF8091A908806696
:107200008093A9088091AB0881FF2CC08091352A1A
:10721000882349F08091AB0884FF05C082E0809309
:10722000AA0881E0AACF9091352A8091342A981734
:10723000A8F4E091352A80912C2A90912D2AE80F0C
:10724000F92FF11D80818093AD088091352A8F5FE1
:107250008093352A83E08093AA08A6CF82E08093AA
:10726000AA088BCF9091362A8091302A981790F4F3
:107270008091AD08E091362A20912E2A30912F2A54
:10728000E20FF32FF11D80838091362A8F5F809368
:10729000362AE0CF86E08093AA0882E06ECF85E0B0
:1072A0006CCF1F920F920FB60F9211242F933F9322
:1072B0008F939F93EF93FF938091A508982F9C70D5
:1072C000E1F08091A50894E082FF93E09093412A39
:1072D0008093A50881E090E08093372A9093382A24
:1072E0001092422AFF91EF919F918F913F912F91A0
:1072F0000F900FBE0F901F90189586FF4EC02091E3
:107300003E2A90913D2A8091A50884FF15C0809166
:107310003A2A882379F083E08093A40885E080935B
:10732000412A1092422A81E090E08093372A90937C
:10733000382AD8CF81E0F0CF80913C2A821790F490
:10734000E0913C2A80913F2A9091402AE80FF92F42
:10735000F11D80818093A80880913C2A8F5F8093E3
:107360003C2AC0CF80913B2A891760F484E090E0EA
:107370008093372A9093382A8091392A81608093AC
:10738000A708B0CF80913A2A882329F083E0809320
:10739000A40881E0C4CF81E0FACF87FF40C090917C
:1073A0003B2A80913D2A9817D8F48091A808E09153
:1073B0003B2A20912A2A30912B2AE20FF32FF11D2C
:1073C000808380913B2A8F5F80933B2A90913D2A56
:1073D00080913B2A8917D8F482E08093A40882CF59
:1073E00080913A2A882389F087E08093A40882E07C
:1073F0008093412A1092422A81E090E08093372ABC
:107400009093382A10923D2A6DCF85E0EECF80917F
:107410003A2A882311F087E0BACF85E0B8CF86E01A
:107420007ECFCF92DF92EF92FF920F931F93CF9375
:10743000DF93A4EFBCE212961D921C92139788EE84
:10744000C82E83E0D82EE12CF12C1496CD92DD923B
:10745000ED92FC92179784EA9EEE8D939C93119780
:1074600020E238E01C962D933C931D971E961C92AB
:107470001E9721E01F962C931F9734E050963C9363
:10748000509752961C92529753961C92539754962B
:107490001C92549755961C9255973BE156963C93F7
:1074A000569757961C92579758961C925897109239
:1074B0008D2D10928E2DE9EAFBE212821382C48296
:1074C000D582E682F7828083918380E698E0848784
:1074D000958788E1868789E1878780E4808B128A97
:1074E000138A148A158A86E2868B178A108E109268
:1074F000422C1092432CE4E4FCE280E89AE0808382
:10750000918312821382148215824AE050E060E077
:1075100070E04683578360877187128613861486CE
:1075200015864FEF5FEF60E070E046875787608B0E
:10753000718BECE5FCE240E059E06DE370E04083E4
:107540005183628373831482158241E050E0468345
:107550005783C4E6DCE28EEB9EEE888399831F821C
:1075600062E06E838CE08A838DE08C838BE08B837A
:1075700038E03D838BEA9DE2FC0112821382C482D3
:10758000D582E682F7820CED1EEE00831183EBEBD1
:10759000FDE21282138270EFE72EF12CE482F58275
:1075A00000E411E006831783E086F18602871387E3
:1075B000168A1486158616861786258B248B0FEF60
:1075C0001FEF028B138B008B118B278B108E118E6C
:1075D000128E15AA29E026AB2AE027AB30AF11AEF8
:1075E00012AE13AE14AE15AE16AE1092FA2D109266
:1075F000FB2D1092FC2D1092FD2DC78FD0A3C4E857
:10760000D4E0C58FD68F33AB24E234E0238F348FA0
:1076100061AB2DEF22AB27EF24AB1092FE2D109221
:10762000FF2D1092002E28E33FEE2083318310922D
:10763000012E1092022EE7EBFDE220E220838183EF
:1076400092831382EFE8FDE288E69FEE80839183C8
:10765000A283B383148215821682178244875587CA
:107660000E94A4086093F02C7093F12C8093F22C6C
:107670009093F32C0E94A408CDEDDCE218821982CD
:107680001A821B821C821D821E821F821886198606
:107690001A860E94A4086B877C878D879E87ECE200
:1076A000EE2EFF24F394EF86F88A04E110E0098BB4
:1076B0001A8BCAECDCE2188219821A821B821C82A5
:1076C0001D821E821F82188619861A860E94A408AF
:1076D0006B877C878D879E87EF86F88A098B1A8B4C
:1076E000EEEBFCE28AE999E9A9E1BEE380839183AC
:1076F000A283B38380E090E0A0EFB2E4848395831B
:10770000A683B783E2EBFCE24DEC5CEC6CE47DE33A
:10771000408351836283738340E050E060E074E40F
:107720004483558366837783E6EAFCE24AE959E9B4
:1077300069E97EE340835183628373838483958305
:10774000A683B783DF91CF911F910F91FF90EF90A8
:10775000DF90CF900895CF93DF93CDB7DEB7EA9750
:10776000CDBFDEBF88ED90E084BF9093610080E0E4
:1077700094E2A4EFB0E08093112890931228A09394
:107780001328B09314288091020686608093020625
:1077900080910006816080930006809102068F7CB4
:1077A000809302068091A0008F788093A000809142
:1077B00002068061809302061092E20581E08093C8
:1077C000E40583E08093010A8FEF90E08093260A1E
:1077D0009093270A80E890E08093380A9093390AC2
:1077E00080933A0A90933B0A80933C0A90933D0A17
:1077F0008BE08093000A8091E50581608093E50528
:107800008091E50582608093E505E0E8FAE037E0E5
:107810002FEF90E885E031832487958780837096E9
:10782000E03C0AE0F007B9F780E094E08093532A47
:107830009093542A8091532A9091542A2FEF30E04C
:10784000B9010E9450506093512A7093522A80913E
:10785000532A9091542AE8EEF3E0BF010E94505061
:1078600060934F2A7093502A8091532A9091542A02
:10787000BF010E94505080934D2A90934E2A20932E
:10788000BC0A3093BD0A8091B50A81608093B50A25
:1078900084E08093B00A8091B00A81608093B00A3E
:1078A00078941092002E40E050E0BA018BEB9DE2FC
:1078B0000E94DF2888E28093022E8093FF2D85E3CB
:1078C0008093FE2D84E38093012E87E890E08093DF
:1078D000032E9093042E80EF90E08093052E9093DA
:1078E000062EE8EEF7E09490E9EEF7E09A941FEFA9
:1078F000911609F47EC014915F0122E0A20EB11C22
:1079000031968490082D0F778BEB9DE20E94131027
:107910008091F22D87FD09C0E091D62DF091D72DF1
:1079200080819091ED2D89238083E091D82DF09175
:10793000D92D80819091EF2D89238083612F8BEB4E
:107940009DE20E94610FE091D82DF091D92D8081A8
:107950009091EE2D892B8083F501D12CC12C10E064
:10796000C016D106FCF48091F02D7F01823089F49D
:107970008091EB2D882369F0DF016D917D917D0170
:107980008BEB9DE20E941C0FEFEFCE1ADE0AF7018F
:10799000E7CFBFEFEB1AFB0A64918BEB9DE20E94ED
:1079A000610FF2CF8091F22D87FD09C0E091D62DB5
:1079B000F091D72D80819091EC2D892B80838BEBDA
:1079C0009DE20E940210F501E00FF11F87FE8ECFAD
:1079D0007F010FEFE01AF00A649170E06F3F7105CC
:1079E00011F464EF71E090E080E00E947408F70108
:1079F0007DCF60E08BEB9DE20E94B31070E060E011
:107A00008BEB9DE20E94C41882E08093CF2D80937F
:107A1000D02D8CE00E94852B91E0811101C090E077
:107A20009093152863E0811101C061E08BEB9DE22A
:107A30000E94B31081E00E94882B62E070E08FE02A
:107A40000E94D20662E070E084E00E94D20662E00A
:107A500070E085E00E94D2068CE090E00E9497558D
:107A60008C0145E064E00E94EA1E0093722A1093A4
:107A7000732A62E070E086E00E94D20682E190E024
:107A80000E949755FC011282138214821582BAE07B
:107A9000CB2ED12CC682D782108614E4E12E1EEEA6
:107AA000F12EE082F18280936E2A90936F2A86E015
:107AB000818BCF010E94140AE0916E2AF0916F2A07
:107AC00002E310E00683178362E070E087E00E9423
:107AD000D20662E070E08CE00E94D2068CE090E07A
:107AE0000E9497555C014CE067E00E94EA1EA0925C
:107AF000682AB092692A62E070E08EE00E94D206A5
:107B000082E190E00E949755FC0112821382148258
:107B10001582C682D7821086E082F18280936C2A19
:107B200090936D2A8EE0818BCF010E94140AE09120
:107B30006C2AF0916D2A068317838BEA9DE20E94DE
:107B4000310E8091B82D9091B92DDC01ED91FC9111
:107B50000688F789E02D6091B72D09958091B82DA1
:107B60009091B92DDC01ED91FC91028CF38DE02D0B
:107B70000995882309F4DFC082E88093BA2D61E07B
:107B800086E00E94150561E085E00E94150561E030
:107B900084E00E94150561E087E00E94150562E01F
:107BA00082E00E94150562E080E00E94150561E018
:107BB00083E00E94150561E081E00E94150582E1E5
:107BC00090E00E949755FC01128213821482158264
:107BD0008AE090E086839783108684E49EEE80831B
:107BE0009183E093612AF093622A8FE0818BCF0129
:107BF0000E94140AE091612AF091622A82E390E0E7
:107C00008683978360914B2811E0612784E00E946E
:107C1000EF0460E087E00E94EF0461E083E00E94EF
:107C2000EF0461E081E00E94EF0460E086E00E94E2
:107C3000EF0460E085E00E94EF041092B02A61E05A
:107C400070E080E10E94D20670E060E080E10E9476
:107C50003A0761E070E081E10E94D20670E060E0E6
:107C600081E10E943A0762E070E082E00E94D20661
:107C700069E670E382E00E94310462E070E083E034
:107C80000E94D20680EA9AE08093442C9093452C7F
:107C90008091A00A8E7F8093A00A1093A60A10926A
:107CA000A10A84E08093A00A80E090E0A4E0B0E024
:107CB0008093582C9093592CA0935A2CB0935B2C02
:107CC0008091A00A8E7F8093A00A8091A00A86707E
:107CD000F0E48F2EF2E49F2EFFE0AF2EB12C853022
:107CE00070F490E0FC01EE0FFF1FE80FF91FE95A56
:107CF000F14180819181A2814C01AA2EB12C950184
:107D000044275527C501B40188279927C12CD12CB8
:107D10007601E394B1E0CB1AD108E108F1086130B3
:107D200071058105910571F4C501B401A7019601A2
:107D30000E94C750EFCF1092BA2D6FEF86E00E94DD
:107D4000AE041DCF60934A2C70934B2C80934C2C27
:107D500090934D2C2093462C3093472C4093482CE5
:107D60005093492CC092522CD092532CE092542C18
:107D7000F092552C611571058105910561F06150F6
:107D800071098109910960934A2C70934B2C80935F
:107D90004C2C90934D2C20934E2C30934F2C409391
:107DA000502C5093512C232B242B252B21F4C090A5
:107DB0004A2CD0904B2CC092AC0AD092AD0A1092B3
:107DC000AA0A1092AB0A8091A00A81608093A00A4F
:107DD0008BED9CE18093562C9093572C81E08093FF
:107DE000A60A8093A50A8091A00A8E7F8093A00A9C
:107DF0008091A00A8670853008F04DC090E0FC01AB
:107E0000EE0FFF1FE80FF91FE85BF141C080D18042
:107E1000E280F12C80E090E0A1E0B0E08093522C71
:107E20009093532CA093542CB093552C9701442736
:107E300055272093462C3093472C4093482C509341
:107E4000492CC701B6018827992760934A2C709363
:107E50004B2C80934C2C90934D2C211531054105D2
:107E60005105C9F1412C512C320163945301420157
:107E7000E1E08E1A9108A108B10861307105810511
:107E8000910589F4C701B601A50194010E94C7506C
:107E900024013501EBCF80E9C82E80EDD82E83E098
:107EA000E82EF12CB7CF60934A2C70934B2C809323
:107EB0004C2C90934D2C4092522C5092532C60920B
:107EC000542C7092552C2093462C3093472C409381
:107ED000482C5093492C8091522C9091532CA09176
:107EE000542CB091552C0197A109B1098093522CC3
:107EF0009093532CA093542CB093552C40914A2C22
:107F000050914B2C60914C2C70914D2C411551058A
:107F10006105710561F04150510961097109409392
:107F20004A2C50934B2C60934C2C70934D2C4091C9
:107F3000462C5091472C6091482C7091492C4093CD
:107F40004E2C50934F2C6093502C7093512C452BFA
:107F5000462B472B21F480914A2C90914B2C8093F7
:107F6000AC0A9093AD0A1092AA0A1092AB0A8091C3
:107F7000A00A81608093A00A8BEE9AE180939D2DE8
:107F800090939E2D10929F2D1092A02D83EF92E33F
:107F90008093A32D9093A42D8CE69BE28093A52D36
:107FA0009093A62D8CE49BE28093A72D9093A82D0F
:107FB00087E59BE28093A92D9093AA2D81E297E219
:107FC0008093A12D9093A22D0091552A1091562AAD
:107FD0008091912D9091922DDC01ED91FC91068480
:107FE000F785E02D42E15AE760E070E009951092D4
:107FF000932D1092942D00939B2D10939C2D0E94F5
:10800000A4086093BA2A7093BB2A8093BC2A9093E9
:10801000BD2A611571058105910511F00E942B5053
:108020008091372881110E94213281E00E94B52B76
:108030000E94A4086093F02C7093F12C8093F22C92
:108040009093F32C80914528909146286091D52AF1
:108050007091D62A8091D72A81110AC081E06115DA
:10806000710509F080E08093D42A81E08093D72ABB
:108070008091D42A86171706A9F087E00E94EF04A2
:108080006091D52A7091D62A81E06115710509F4B5
:1080900080E08093D42A80914B28882319F081E1D5
:1080A0000E943A078091D32A882309F48DC0109248
:1080B000D32A8091452890914628892B29F08091D8
:1080C000E32A882309F46DC02091162830911728DF
:1080D0006091582A7091592A80915A2A90915B2A6E
:1080E000032E000C440B550B0E94C7506093582A76
:1080F0007093592A80935A2A90935B2A8091E42C9A
:108100009091E52C0197029708F053C0E091402828
:10811000F0914128CF010A9608E010E0B8010E94D2
:1081200045559C01220F331F2F57354DCF0109961E
:10813000B8010E944555FC01EE0FFF1FEF57F54DAA
:10814000D9018D919C9120813181821B930B865A9C
:108150009F4F80931628909317288091E42A8823B4
:10816000C1F08091572A22EE3FEF811102C02EE12B
:1081700030E08091162890911728820F931F8093EA
:108180001628909317288091572A91E08927809389
:10819000572A8091B22A882379F01092B22A0E943D
:1081A000752780E090E0892B09F442CF0E940000FF
:1081B0003FCF90E080E0CBCF80914B28882389F39C
:1081C00081E08093B32AEDCF8091D22A882319F0E1
:1081D0000E941228E6CF8091D12A882381F10E9443
:1081E0001228609138287091392880913A2890910E
:1081F0003B280E94DE530E94DC516B017C011C1461
:108200001D041E041F046CF68091CF2A9091D02A81
:108210008C33910554F08C199D0997FF03C09195FB
:108220008195910903970CF4BCCF40E0C701B601DA
:108230000E949820C092CF2AD092D02AB2CF8091AB
:10824000C72A81110DC00E94A4086093C32A7093AD
:10825000C42A8093C52A9093C62A81E08093C72AB6
:108260004091C32A5091C42A6091C52A7091C62AB0
:108270004115510561057105E1F08091F02C909157
:10828000F12CA091F22CB091F32C841B950BA60B32
:10829000B70B813D9740A105B10558F080E00E94E1
:1082A0004D231092C32A1092C42A1092C52A10920C
:1082B000C62A8091912D9091922DDC01ED91FC9137
:1082C0000084F185E02D0995181619060CF074C08C
:1082D0008091912D9091922DDC01ED91FC91028481
:1082E000F385E02D0995282F8091932D9091942D61
:1082F0008130910509F49EC18230910509F4AFC126
:10830000892B09F059C088E0820F8530A0F1409197
:108310009B2D50919C2D4115510541F0822F8F705E
:1083200090E001964817590709F046C0822F203F78
:1083300008F4807F8093982D883FD1F1F0F4803944
:1083400049F1803B91F18091912D9091922DDC012A
:10835000ED91FC910190F081E02D622F09958091C3
:10836000912D9091922DDC01ED91FC910680F78189
:10837000E02D099521C0822FDDCF8B3F09F455C137
:108380008C3F09F44DC18A3FF1F68FE89DE20E94CF
:10839000851A12C081E090E08093952D9093962DE0
:1083A0008093932D9093942D07C081E090E0F8CFB7
:1083B0008FE89DE20E948D1A0091612A1091622A35
:1083C000F801808580FD15C00E94A408D801199687
:1083D000CD90DD90ED90FC901C976C197D098E0975
:1083E0009F0960935D2A70935E2A80935F2A909321
:1083F000602AC0905D2AD0905E2AE0905F2AF090BB
:10840000602AC8010E94AB0980915C2A811152C187
:108410008091612A9091622A0E94A309811107C06C
:10842000B8ECCB16D104E104F1040CF443C1809103
:108430003728882309F42FC10E94A4086093BA2A20
:108440007093BB2A8093BC2A9093BD2A8091B92A4D
:10845000882309F420C180E00E94B52B8091C12AB5
:108460009091C22A01968093C12A9093C22A6BE010
:1084700070E00E944555892B99F483E00E94FE0725
:108480009C0191E02115310509F090E080911828B8
:10849000981731F090931828232B11F40E94C127CC
:1084A0008091C12A9091C22A67E070E00E944555F0
:1084B000892BD1F58091722A9091732A0E94D61E41
:1084C0006B01A090E42CB090E52CF2E0AF1AB1085B
:1084D0006090D12C7090D22C02E0601A710800914B
:1084E000702A1091712A0617170709F4BDC1CB0134
:1084F00081709927892B09F0B7C18091372888238B
:1085000009F445C10E94A4086093BA2A7093BB2A5B
:108510008093BC2A9093BD2A8091B92A882309F4BC
:1085200036C180E00E94B52B809145289091462865
:10853000892B09F0DBC38091C12A9091C22A6DE09A
:1085400070E00E9445558C01892B09F0CFC38091C2
:10855000792A811105C00E94A40881E08093792ABC
:1085600085E10E9423081C0126E0221A310860E000
:1085700074E0681B790B072E000C880B990B36EF03
:10858000231633E0330608F490C30E9414526B01A3
:108590007C01C092B62CD092B72CE092B82CF0920D
:1085A000B92CC092752AD092762AE092772AF0925E
:1085B000782A8091742A882309F454C584E1E0EC78
:1085C000FDEEDE01559601900D928A95E1F784E16A
:1085D000E4EDFDEEDE01119601900D928A95E1F732
:1085E00020E030E040EA50E4C701B6010E94655146
:1085F00087FD2EC520E030E44EE754E4C701B60104
:108600000E941C534E0149E1840E911C18160CF077
:1086100026C4A8E88A2EA3E19A2EA12CB12C1DC550
:108620008FE89DE20E947D1AC7CE8FE89DE20E94EE
:10863000751AC2CE8091982D803939F0803B51F067
:108640001092932D1092942DB7CE27FDF9CF209341
:10865000972D02C027FFFBCF82E090E0A1CE809152
:10866000982D803971F0803B59F7E091A12DF09160
:10867000A22D309729F3422F6091972D81E0099523
:10868000DFCF27FDDDCF4091972D61E08FE89DE2A0
:108690000E94951AD5CF81E080935C2A80914B2867
:1086A0008823F9F0E8ECCE16D104E104F104CCF40F
:1086B0000E94C12780915C2A882309F4CFCEE091E3
:1086C000612AF091622A808580FFC8CE10925C2AD0
:1086D00010925D2A10925E2A10925F2A1092602AF0
:1086E000BDCE11E060E081270E94172B80914B28BE
:1086F000882309F442C01092D52A1092D62A60E04D
:1087000087E00E94EF048091452890914628892BAC
:1087100059F5E091442CF091452C80818E7F808327
:10872000168380818E7F808316838091462C909162
:10873000472CA091482CB091492C80934E2C9093BB
:108740004F2CA093502CB093512C892B8A2B8B2B20
:1087500079F08091522C9091532C848795871286C2
:10876000138680818160808381E08093B22AA2CFCA
:1087700080914A2C90914B2CF0CF2091452830913C
:10878000462881E02130310581F380E0EECFC6013B
:10879000801B910B21E030E01816190614F02FEF22
:1087A0003FEF12E0A116B10408F0CDC08091952AE8
:1087B0009091962A08964091932A5091942A841B6E
:1087C000950B68E070E00E944555AC01DC01AA0FF2
:1087D000BB1FFD01EF57F54D00811181F80117FF17
:1087E00007C0EE27FF27E01BF10B319521953109DA
:1087F0002130310549F4E531F1054CF4E830F1055B
:1088000044F52E0F3F1F0FC0E631F105FCF0C90102
:10881000880F991F280F391F2E0F3F1F2F31310549
:1088200014F02EE130E017FF03C031952195310996
:10883000AF57B54D2D933C9380914B28882361F021
:10884000BA0181E090E00E94B0080AC0E930F10569
:10885000C4F2220F331FD5CF61E080E00E942721B0
:10886000C092702AD092712A80916E2A90916F2ABC
:108870000E94AB0980916C2A90916D2A0E94AB09ED
:1088800080916E2A90916F2A0E94A309182F8091DF
:108890006C2A90916D2A0E94A309982E1123C9F089
:1088A00080913728882371F00E94A4086093BA2A27
:1088B0007093BB2A8093BC2A9093BD2A8091B92AD9
:1088C00081112FCE80916B2A882309F49BC01092CE
:1088D0006B2A8091682A9091692A0E94D61E6B01AA
:1088E0000091662A1091672A0617170709F4FDC040
:1088F000CB0181709927892B09F0F7C08091372827
:10890000882371F00E94A4086093BA2A7093BB2A4E
:108910008093BC2A9093BD2A8091B92A811101CEFF
:10892000C601801B910B181619060CF0B2C081E02D
:1089300090E02091952A3091962A820F931F97FFFD
:10894000ABC00896FCCF42E06416710408F045C045
:108950008091952A9091962A08964091932A509159
:10896000942A841B950B68E070E00E944555AC0189
:10897000FC01EE0FFF1FDF01AF5DB74D8D919C91A4
:10898000280F391F29833A8381E090E08D8B9E8BDD
:10899000DE0122303105D4F0119688E090E089A7FD
:1089A0009AA78D919C911197089714F0DE019996E2
:1089B000EF5DF74D8D919C918083918380914B2841
:1089C000882331F0BA0182E090E03DCF5596E5CFA3
:1089D00061E080E00E94C12143CF8091E72A90911D
:1089E000E82A820F931F97FF02C00A96FCCF6AE025
:1089F00070E00E9445558093E72A9093E82A0E94F0
:108A0000DA1F2ECF52E0A516B104E0F48091952A2A
:108A10009091962A08962091932A3091942A821B4D
:108A2000930B68E070E00E944555FC01EE0FFF1FBC
:108A3000EF57F54D10821182AC0160E080E00E949A
:108A4000272147CF82E068167104F0F48091952ABF
:108A50009091962A08962091932A3091942A821B0D
:108A6000930B68E070E00E944555FC01EE0FFF1F7C
:108A7000EF5DF74D21E030E020833183AC0160E011
:108A800080E00E94C12125CF10926A2A0E946826A8
:108A900020CF8FEF9FEF4DCF877099278093952A36
:108AA0009093962AA2E0AA16B10408F08CC008960A
:108AB0002091932A3091942A821B930B68E070E0F6
:108AC0000E94455520914B28222331F0BC0181E0C2
:108AD00090E00E94B00805C0AC0161E080E00E9417
:108AE0002721C092662AD092672AE2E0AE16B1042E
:108AF00008F44CC0F2E06F16710408F447C080918E
:108B0000452890914628019709F440C08091652A34
:108B100081113CC000916C2A10916D2AD8011896E1
:108B20008C9180FD33C00E94A408F8010185128554
:108B300023853485601B710B820B930B653F71405D
:108B40008105910518F181E08093652A8091632A5F
:108B50009091642A0196833091050CF06BC080934C
:108B6000632A9093642AE091632AF091642AEE0FBD
:108B7000FF1FEE0FFF1FEA59F14160817181828171
:108B800093810E94DC51CB010E948324992009F437
:108B9000CBCC80913728882371F00E94A408609381
:108BA000BA2A7093BB2A8093BC2A9093BD2A8091E5
:108BB000B92A8111B6CC8091652A882309F43FC077
:108BC0001092652AB1CCB2E06B167104C8F4089615
:108BD0002091932A3091942A821B930B68E070E0D5
:108BE0000E94455520914B28222321F0BC0182E0B0
:108BF00090E06FCFAC0161E080E00E94C12171CFB5
:108C000049E150E063E070E084E890E00E94151BC9
:108C10008091952A9091962A01960E94FB208FEFD1
:108C20009FEF8093CD2D9093CE2D8093CB2D90935D
:108C3000CC2D57CF1092632A1092642A94CF02E071
:108C4000A016B10408F470CC12E06116710408F4A7
:108C50006BCC8091952A9091962A019689839A836C
:108C600021E030E02D8B3E8BFE010297E4F031963F
:108C700088E090E089A79AA780819181089714F0F5
:108C8000FE01B9968081918120913E2830913F2844
:108C90008217930709F448CC80933E2890933F288D
:108CA0000E94372341CC7596E3CF0E941452AB014A
:108CB000BC0182EB9CE20E943B1D6B017C01209178
:108CC000752A3091762A4091772A5091782A0E940D
:108CD000F8500E94DC519B0177FF04C02227332704
:108CE000261B370B233031050CF05BCC8091C12A59
:108CF0009091C22A6BEB70E00E944555892B11F4CC
:108D00000E94B62F2091C12A3091C22AC90165E282
:108D100070E00E944555892B09F084C34DED5CE25B
:108D20006AEC7CE282E090E00E94EB08182F882336
:108D3000C1F18091D12C9091D22C0297029788F5A5
:108D40008091D02C882311F181E090E0809321283C
:108D50009093222880932328909324288093252879
:108D60009093262880932728909328288093292859
:108D700090932A2880932B2890932C2880932D2839
:108D800090932E2880932F289093302880914B2801
:108D9000882309F494C26FEF7FEF82E090E00E9495
:108DA000B0084AEC5CE26DED7CE290E080E00E946D
:108DB000EB08882309F49FC68091E42C9091E52C60
:108DC0000297029778F58091E32C882301F11092A5
:108DD000812A1092822A1092832A1092842A109259
:108DE000852A1092862A1092872A1092882A109239
:108DF000892A10928A2A10928B2A10928C2A109219
:108E00008D2A10928E2A10928F2A1092902A809189
:108E10004B28882309F45AC26FEF7FEF81E090E07E
:108E20000E94B00880913728882309F456C20E9416
:108E3000A4086093BA2A7093BB2A8093BC2A9093AB
:108E4000BD2A8091B92A882309F447C280E00E9494
:108E5000B52BA7C985010430110509F48FC058014D
:108E60005FEFA51AB50AF40181919191A191B19199
:108E70004F018FA798ABA9ABBAABBC01CD010E9443
:108E80001452A70196010E941C5318161CF7AA0C35
:108E9000BB1CAA0CBB1CE1E0F0E0EC0FFD1FEA0DCF
:108EA000FB1D40805180628073805801AA0CBB1C5E
:108EB000AA0CBB1C88248394912C8C0E9D1EA80C9C
:108EC000B91CD5016D917D918D919C910E94145298
:108ED0000E94DC516BA77CA78DA79EA7D501549655
:108EE0000D911D912D913C9157970FAB18AF29AF64
:108EF0003AAFC301B2010E9414520E94DC514B01EF
:108F00005C010BA51CA52DA53EA5801A910AA20AFD
:108F1000B30A8BAA9CAAADAABEAAC701B6010E9439
:108F2000DC518FA898ACA9ACBAAC681979098A0948
:108F30009B092BA93CA94DA95EA90E9429552FA5E3
:108F400038A949A95AA9281939094A095B090E946F
:108F500064508BA49CA4ADA4BEA4820E931EA41E38
:108F6000B51E8BA69CA6ADA6BEA6481459046A04DD
:108F70007B0424F44BA65CA66DA67EA66BA57CA5FF
:108F80008DA59EA50E94145206EF201603E0300620
:108F900008F4AFC06093AA2C7093AB2C8093AC2CD8
:108FA0009093AD2C0E94DC512091472830914828A5
:108FB0002617370709F46BC1609347287093482838
:108FC0008093492890934A280E9414526FA778AB47
:108FD00089AB9AAB8090312890903228A0903328AA
:108FE000B09034288BAA9CAAADAABEAA9B01AC0162
:108FF00060EC71EE84E69CE40E946A51A501940144
:109000000E94215320E030E044EB52E40E946A5178
:109010000E94DE530E94E3516B017C010091442CBD
:109020001091452CD8018C918E7F8C938C918670F9
:10903000823009F4ABC0843009F464C0811169C086
:1090400054E0CC0CDD1CEE1CFF1C5A95D1F761C01E
:10905000BEE18B2E912CA12CB12C8BA69CA6ADA68B
:10906000BEA68CCFC701B6010E94DC519B01AC01AA
:109070002550310941095109A4E5B1E00E9483500E
:1090800027EF33E040E050E00E946450CA01B9018C
:10909000675E7F4F8F4F9F4F0E9414526B017C0180
:1090A00020E030E040EF51E40E941C5318169CF47D
:1090B00020E030E044EB53E4C701B6010E94655163
:1090C00087FF10C0C701B6010E94DC516BA77CA7C7
:1090D0008DA79EA753CFC12CD12CF0EFEF2EF1E43A
:1090E000FF2EF0CFC12CD12CE4EBEE2EE3E4FE2ECC
:1090F000E9CFAB01BC0186EA9CE20E943B1D0E94C5
:109100004F5250CF72E0F694E794D794C7947A9573
:10911000D1F7812C912C5401A3948092522C9092DF
:10912000532CA092542CB092552C970144275527CC
:109130002093462C3093472C4093482C5093492C35
:10914000C701B6018827992760934A2C70934B2C4E
:1091500080934C2C90934D2C2115310541055105E0
:10916000A9F124013501A1E04A1A510861087108EA
:10917000613071058105910589F4C701B601A3012C
:1091800092010E94C75053014201EBCF63E0CC0C27
:10919000DD1CEE1CFF1C6A95D1F7BBCF60934A2CF7
:1091A00070934B2C80934C2C90934D2C8092522C8E
:1091B0009092532CA092542CB092552C2093462C74
:1091C0003093472C4093482C5093492C8091522C3B
:1091D0009091532CA091542CB091552C0197A1093A
:1091E000B1098093522C9093532CA093542CB0939C
:1091F000552C40914A2C50914B2C60914C2C7091E5
:109200004D2C411551056105710561F04150510921
:109210006109710940934A2C50934B2C60934C2C5C
:1092200070934D2C4091462C5091472C6091482CC6
:109230007091492C40934E2C50934F2C6093502C9E
:109240007093512C452B462B472B21F480914A2CAF
:1092500090914B2CF8018487958712861386808124
:10926000816080838091452890914628892B79F4EC
:109270002BA93CA94DA95EA96FA578A989A99AA98E
:109280000E946A510E94DC5140E00E949820809127
:109290003728882309F42ACD0E94A4086093BA2AAB
:1092A0007093BB2A8093BC2A9093BD2A8091B92ADF
:1092B000882309F41BCD80E00E94B52B17CD50E028
:1092C00040E061E081E00E94C1216BCD50E040E0D0
:1092D00061E081E00E942721A5CD61E08091D12C41
:1092E0009091D22C019709F460E083E00E94EF0492
:1092F00061E08091E42C9091E52C019709F460E005
:1093000081E00E94EF048091D12C9091D22C0297A1
:10931000029738F08091E42C9091E52C0297029707
:1093200050F58091952A9091962A8093932A909354
:10933000942A8091D12C9091D22C0297029740F4DC
:109340008AEC9CE20E94AA1A682F83E00E94EF0434
:109350008091E42C9091E52C0297029710F00C94E8
:10936000D1408DED9CE20E94AA1A682F81E00E94F4
:10937000EF040C94D14080914B28882309F446C017
:1093800080915C2890915D28A0915E28B0915F2823
:10939000892B8A2B8B2B51F40E94A40860935C28A4
:1093A00070935D2880935E2890935F2881E080937E
:1093B00062288091D12C9091D22C0297029770F064
:1093C0008091D32C9091D42C0297029738F48091FD
:1093D0004B28882309F181E08093922A8091E42C24
:1093E0009091E52C0297029708F4A3CF8091E62C88
:1093F0009091E72C0297029708F09BCF80914B2821
:10940000882369F081E08093912A93CF81E00E94C4
:109410004D230E94DA1FCDCF0E94F52ADFCF0E9494
:10942000062B87CFC90165E370E00E944555892B63
:10943000C9F480915C2890915D28A0915E28B0913C
:109440005F28892B8A2B8B2B69F00E94A40820911E
:109450005C2830915D28621B730B6D32714014F0F3
:109460000E94E0238091C02A811134C1312C809167
:10947000C12A9091C22A60E177E20E944555892B6A
:10948000A9F480914B28882309F4A9C18091F02C7C
:109490009091F12CA091F22CB091F32C8093BA2AE8
:1094A0009093BB2AA093BC2AB093BD2A8091B92A7D
:1094B000882309F4E3C08091B52A9091B62AA0913F
:1094C000B72AB091B82A4091F02C5091F12C6091BC
:1094D000F22C7091F32C481B590B6A0B7B0B4F310C
:1094E00051056105710508F4C9C04E96A11DB11D55
:1094F0008093B52A9093B62AA093B72AB093B82A3E
:1095000080913728882309F4B9C06091A72A709107
:10951000A82A072E000C880B990B0E9414526B018D
:109520007C016091C52D7091C62D072E000C880B13
:10953000990B0E9414529B01AC01C701B6010E9415
:109540006A512B013C0120911D2830911E28409129
:109550001F28509120280E948E534B015C010091DE
:10956000A52A1091A62AC090A12AD090A22AE09004
:109570001B28F0901C2860919F2A7091A02A6C19DA
:109580007D09072E000C880B990B0E941452A30131
:1095900092010E9421532B013C01B601DD0C880B86
:1095A000990B0E9414529B01AC01C301B2010E94AD
:1095B000F9500E94DC512B016091A32A7091A42ADA
:1095C000601B710B072E000C880B990B0E94145224
:1095D000A50194010E9421534B015C01B801110FB8
:1095E000880B990B0E9414529B01AC01C501B40178
:1095F0000E94F9500E94DC5140919D2A50919E2A70
:10960000E0919B2AF0919C2A82019B01BF018BEB88
:109610009DE20E944C188091192890911A2820915F
:10962000A72A3091A82A280F391F2093A72A309300
:10963000A82A4091C52D5091C62D840F951F8217E1
:109640009307E4F48091992A90919A2A01962091A7
:10965000972A3091982A2F5F3F4F2093972A309373
:10966000982A64E070E00E9445558093992A90936F
:109670009A2A8091372881110E9421328091C02A34
:1096800010E000E0882309F4D9C0E091BE2AF091EF
:10969000BF2A628587E00E94EF048091BE2A9091E4
:1096A000BF2ADC011A962C91222311F03110BEC082
:1096B00090E080E00E9437238091B42A811104C099
:1096C00090E080E00E943F2281E08093B42A0FEF77
:1096D0001FEFB4C00091BE2A1091BF2A0E94A408B7
:1096E0002B013C01D80114968C9130E020E08B32A4
:1096F00018F40E94FE079C0191E02130310509F425
:1097000090E0F801928786810E9423082FEF33E0D2
:10971000281B390BD80118962D933C9319971A964C
:109720003C90F80131100DC01786108A118A128AF8
:109730008FEF9FEF838B948B85879687108611869A
:1097400096CE87859089A189B289892B8A2B8B2B0C
:1097500021F44786508A618A728AF801E384F4848E
:10976000E586F686C8010E943624D8011B968D93A3
:109770009C931C971F964D915D916D917C91529792
:10978000411551056105710509F470CE441A550A59
:10979000660A770A55962D913C915697032E000C38
:1097A000440B550B241535054605570508F05ECECC
:1097B00053962D913C918217930709F457CEE816E2
:1097C000F90609F053CEF8011786108A118A128A19
:1097D000E38AF48A8FEF9FEF8587968748CE809142
:1097E0003728882309F462CE8091B92A811163CE8B
:1097F0000E94A4080091BA2A1091BB2A2091BC2A89
:109800003091BD2A601B710B820B930B613E734933
:109810008440910508F432CF81E08093B92A70E04A
:1098200060E08BEB9DE20E94C41840CE0E9436247B
:109830008C0181E08093B32A1092B42A8091B22ADD
:10984000882321F01092B32A0C94D1408091D12A20
:1098500081110C94D14080914B2881110AC08091D4
:10986000C02A811106C08091B12A882311F40C947A
:10987000D1408091B32A8823E9F08091B02A8823CF
:1098800031F060E085E00E94EF041092B02A10925F
:10989000B32A81E08093AF2A8091B12A882309F40A
:1098A0005BC060E080913528909136280E94DE22CE
:1098B0000E94E023609147287091482880914928B0
:1098C00090914A2822E030E040E050E00E9464504D
:1098D000CA01B9010E9414522091312830913228D6
:1098E00040913328509134280E946A5120E030E49E
:1098F0004CE955E40E941C5308EC10E087FF02C0BD
:1099000008E512E08091AF2A882311F40C94D1402D
:109910000E944508AB01BC01C801110FAA0BBB0B8B
:109920000091AB2A1091AC2A2091AD2A3091AE2A39
:10993000800F911FA21FB31F481759076A077B07A3
:1099400010F40C94D1401092AF2A70E060E080E1F6
:109950000E943A070C94D140D090C02ADD2019F023
:1099600060E0C801A3CFE0903E28F0903F288091AE
:10997000A92A9091AA2A01978093A92A9093AA2AAA
:109980000091402810914128181619060CF455C072
:1099900080913C2890913D288330910509F479C04D
:1099A000A8F4009140281091412881309105F1F0F0
:1099B000029769F100914028109141280F5F1F4FD5
:1099C0000E151F05ACF110E000E032C084309105A7
:1099D00009F475C0059771F70E94804F892F990F80
:1099E000990BB7010E9445558C0127C00150110900
:1099F000C701019717FD03C00E151F050CF08C0160
:109A0000DD24D39480179107C1F0D12C16C080912A
:109A10004228882391F10F5F1F4F17FF31C081E06B
:109A20008093422810E000E0D0904228DD2029F009
:109A3000DD24D3940115110541F76D2DC8010E9455
:109A4000DE228091A92A9091AA2A181619060CF4F0
:109A50002FCF8091D12C9091D22C0197029708F0B2
:109A600047C0000F111FF801EF5DF74D8081918114
:109A70008093A92A9093AA2A1BCF01501109CDCF18
:109A80000E151F058CF28701015011091092422812
:109A9000CBCFB1E0EB16F10409F495CF80914028CB
:109AA000909141288C010E5F1F4F0E151F050CF47D
:109AB000BFCF8C010095109501701127B9CF80910F
:109AC0004328909144280196B7010E944555809300
:109AD000432890934428FC01EE0FFF1FE45BF74DF1
:109AE00000811181DD24D394892B09F4A6CF8DCF79
:109AF00081E090E0BDCF111195C91BCCCF93DF93CE
:109B0000DC012D91FB013191EC013883EB012883BD
:109B100041505109CD01BF01141615068CF3DF9198
:109B2000CF910895B0E0A0E0E8E9FDE40C94A050E6
:109B30006C01D62FC72F8A017901F9010995B80167
:109B400097FF15C08D2F9C2FF701099597FD08C031
:109B5000B801C601F701099597FD16C0DC2DCD2D82
:109B60008D2F9C2FCDB7DEB7E8E00C94B9508D2F28
:109B70009C2FF70109951816190694F3B801C60130
:109B8000F701099597FDEACFD02FC12FE9CFA8E0C3
:109B9000B0E0EDECFDE40C9496508C014F835887B7
:109BA00059019A013195219531092D833E836F80AA
:109BB0007884600E711E6730710578F58F81988505
:109BC000689F6001699FD00C789FD00C1124C00E53
:109BD000D11E6C147D0420F02896E2E10C94AF5065
:109BE000730113C047012F813885821A930AB70188
:109BF000C401F50109951816190654F44F815885CA
:109C0000B401C7010E947E4D74010E151F0550F36B
:109C1000EF81F8856E0E7F1EDCCFCB019695879580
:109C20002F813885829F6001839FD00C929FD00C3A
:109C30001124C00ED11ECB010197829F1001839F7A
:109C4000300C929F300C11247801E20CF31C673029
:109C5000710509F442C0C701280169327105B0F1EC
:109C600083E0769567958A95E1F7629F4001639F4F
:109C7000900C729F900C1124C401880F991F898346
:109C80009A83AC01400F511FB801680D791D9501F1
:109C9000C8010E94924D2C01A601480D591D9194B6
:109CA000819491089501B601C601880D991D0E9405
:109CB000924D6C01B701680D791D9501A701C7018F
:109CC000E981FA818E1B9F0B0E94924D9501AC0198
:109CD000B601C2010E94924D6C014F815885B601B8
:109CE000C8010E947E4D43016301270119821A8237
:109CF000EC14FD0408F446C0B801C601F50109954D
:109D00001816190654F1892B71F44F815885B60144
:109D1000C3010E947E4D2F813885620E731E81E043
:109D200090E089839A83EF81F885CE0EDF1EE0CF25
:109D3000892B71F44F815885B201C7010E947E4D75
:109D40002D813E81420E531E81E090E089839A83EB
:109D5000EB80FC80EC14FD04A8F0B801C701F5010C
:109D600009952D813E812E0D3F1D2B833C8397FF4E
:109D7000DFCF4F815885B701C6010E947E4DEB8031
:109D8000FC80CDCFEF81F8852E0E3F1E200E311EB8
:109D900029813A81232B09F58214930408F01CCF02
:109DA000740113C06701EF81F885CE1ADF0AB7018D
:109DB000C601F50109951816190654F44F81588506
:109DC000B601C7010E947E4D76010E151F0550F3A6
:109DD0008F819885880E991EDFCF460186189708D7
:109DE000A301401B510B841695060CF4A401141614
:109DF000150634F4B601641B750BC8010E947E4D34
:109E000092012E193F097901A101441955098F8149
:109E10009885481B590B2417350708F4A901141617
:109E2000150634F4B101641B750BC6010E947E4D0A
:109E3000EF81F885E815F90548F4C401BF010E94D7
:109E400050509501AF01C8010E94C74D2F81388540
:109E50002E153F0508F0C0CE81010E191F09C7015C
:109E6000B9010E945050A3CE8F929F92AF92BF92A1
:109E7000CF92DF92EF92FF92CF93DF93EC01688154
:109E800079818A819B81611571058105910521F494
:109E900064E279ED8BE597E02DE133EF41E050E0AE
:109EA0000E94645049015A019B01AC01A7EAB1E448
:109EB0000E9483506B017C01ACEEB4EFA5019401CC
:109EC0000E949150DC01CB018C0D9D1DAE1DBF1D6C
:109ED000B7FF03C00197A109B04888839983AA837B
:109EE000BB839F77DF91CF91FF90EF90DF90CF9072
:109EF000BF90AF909F908F9008950E94344F089527
:109F000087E698E20E94344F0895B0E0A0E0809385
:109F1000672890936828A0936928B0936A280895C9
:109F20008F929F92AF92BF92CF92DF92EF92FF9269
:109F3000CF93DF93EC01688179818A819B816115E0
:109F400071058105910521F464E279ED8BE597E0D7
:109F50002DE133EF41E050E00E94645049015A0185
:109F60009B01AC01A7EAB1E40E9483506B017C0124
:109F7000ACEEB4EFA50194010E949150C60ED71E1D
:109F8000E81EF91EF7FE06C081E0C81AD108E108F4
:109F900080E8F80AC882D982EA82FB82C701B6014A
:109FA0009F77DF91CF91FF90EF90DF90CF90BF90A0
:109FB000AF909F908F9008958F929F92AF92BF9293
:109FC000CF92DF92EF92FF9260916B2870916C2894
:109FD00080916D2890916E2861157105810591051C
:109FE00021F464E279ED8BE597E02DE133EF41E078
:109FF00050E00E94645049015A019B01AC01A7EA5C
:10A00000B1E40E9483506B017C01ACEEB4EFA5017A
:10A0100094010E949150C60ED71EE81EF91EF7FE4D
:10A0200006C081E0C81AD108E10880E8F80AC092A9
:10A030006B28D0926C28E0926D28F0926E28C701B0
:10A04000B6019F77FF90EF90DF90CF90BF90AF90D9
:10A050009F908F90089560936B2870936C288093E5
:10A060006D2890936E28089503D0808199270895D4
:10A07000FC01E050FC4E0895262FAF93BF93E0E023
:10A08000F0E1328131FDFDCFDC01A050BC4E2C93BC
:10A090002DE924BF23E020830196BF91AF9108955D
:10A0A000AA1BBB1B51E107C0AA1FBB1FA617B707FE
:10A0B00010F0A61BB70B881F991F5A95A9F780951A
:10A0C0009095BC01CD010895052E97FB1EF40094D8
:10A0D0000E947B5057FD07D00E94C75007FC03D059
:10A0E0004EF40C947B5050954095309521953F4F00
:10A0F0004F4F5F4F089590958095709561957F4F74
:10A100008F4F9F4F08950E94E950A59F900DB49FD7
:10A11000900DA49F800D911D11240895B7FF0C94FC
:10A1200083500E948350821B930B08952F923F927D
:10A130004F925F926F927F928F929F92AF92BF9257
:10A14000CF92DF92EF92FF920F931F93CF93DF9303
:10A15000CDB7DEB7CA1BDB0BCDBFDEBF09942A88A3
:10A16000398848885F846E847D848C849B84AA842B
:10A17000B984C884DF80EE80FD800C811B81AA81B8
:10A18000B981CE0FD11DCDBFDEBFED010895A1E293
:10A190001A2EAA1BBB1BFD010DC0AA1FBB1FEE1F61
:10A1A000FF1FA217B307E407F50720F0A21BB30BAC
:10A1B000E40BF50B661F771F881F991F1A9469F728
:10A1C00060957095809590959B01AC01BD01CF0184
:10A1D0000895A29FB001B39FC001A39F700D811D80
:10A1E0001124911DB29F700D811D1124911D0895A0
:10A1F0005058BB27AA270E9410510C94CA520E94A3
:10A20000BC5238F00E94C35220F039F49F3F19F439
:10A2100026F40C94B9520EF4E095E7FB0C948A52A4
:10A22000E92F0E94DB5258F3BA17620773078407BD
:10A23000950720F079F4A6F50C9415530EF4E095EB
:10A240000B2EBA2FA02D0B01B90190010C01CA01F0
:10A25000A0011124FF27591B99F0593F50F4503E9B
:10A2600068F11A16F040A22F232F342F4427585F8D
:10A27000F3CF469537952795A795F0405395C9F7A5
:10A280007EF41F16BA0B620B730B840BBAF091505D
:10A29000A1F0FF0FBB1F661F771F881FC2F70EC0FC
:10A2A000BA0F621F731F841F48F4879577956795CF
:10A2B000B795F7959E3F08F0B0CF9395880F08F0BB
:10A2C0009927EE0F9795879508950E94665208F496
:10A2D00081E008950E947E510C94CA520E94C3529C
:10A2E00058F00E94BC5240F029F45F3F29F00C94D2
:10A2F0008A5251110C9416530C94B9520E94DB529D
:10A3000068F39923B1F3552391F3951B550BBB27A4
:10A31000AA2762177307840738F09F5F5F4F220FE9
:10A32000331F441FAA1FA9F335D00E2E3AF0E0E8E0
:10A3300032D091505040E695001CCAF72BD0FE2F2A
:10A3400029D0660F771F881FBB1F261737074807BE
:10A35000AB07B0E809F0BB0B802DBF01FF27935876
:10A360005F4F3AF09E3F510578F00C948A520C945E
:10A3700016535F3FE4F3983ED4F38695779567953F
:10A38000B795F7959F5FC9F7880F911D96958795AB
:10A3900097F90895E1E0660F771F881FBB1F6217CA
:10A3A00073078407BA0720F0621B730B840BBA0B88
:10A3B000EE1F88F7E09508950E94E3516894B1116B
:10A3C0000C94165308950E94E35288F09F5798F01A
:10A3D000B92F9927B751B0F0E1F0660F771F881FAA
:10A3E000991F1AF0BA95C9F714C0B13091F00E94C4
:10A3F0001553B1E008950C941553672F782F8827D3
:10A40000B85F39F0B93FCCF3869577956795B395EA
:10A41000D9F73EF490958095709561957F4F8F4F59
:10A420009F4F0895E89409C097FB3EF4909580955E
:10A43000709561957F4F8F4F9F4F9923A9F0F92F0A
:10A4400096E9BB279395F695879577956795B79588
:10A45000F111F8CFFAF4BB0F11F460FF1BC06F5F6E
:10A460007F4F8F4F9F4F16C0882311F096E911C080
:10A47000772321F09EE8872F762F05C0662371F0A1
:10A4800096E8862F70E060E02AF09A95660F771FB5
:10A49000881FDAF7880F9695879597F908950E9497
:10A4A000FD5290F09F3748F4911116F00C9416531A
:10A4B00060E070E080E89FEB089526F41B16611DB4
:10A4C000711D811D0C9490520C94AB52990F000891
:10A4D000550FAA0BE0E8FEEF16161706E807F90776
:10A4E000C0F012161306E407F50798F0621B730B11
:10A4F000840B950B39F40A2661F0232B242B252B92
:10A5000021F408950A2609F4A140A6958FEF811D34
:10A51000811D089597F99F6780E870E060E00895D5
:10A52000882371F4772321F09850872B762F07C06A
:10A53000662311F499270DC09051862B70E060E0DE
:10A540002AF09A95660F771F881FDAF7880F96957D
:10A55000879597F908959F3F31F0915020F48795A2
:10A5600077956795B795880F911D9695879597F97B
:10A5700008959FEF80EC089500240A94161617069C
:10A5800018060906089500240A94121613061406E4
:10A5900005060895092E0394000C11F4882352F047
:10A5A000BB0F40F4BF2B11F460FF04C06F5F7F4FFF
:10A5B0008F4F9F4F089557FD9058440F551F59F0E6
:10A5C0005F3F71F04795880F97FB991F61F09F3FA0
:10A5D00079F087950895121613061406551FF2CFC9
:10A5E0004695F1DF08C0161617061806991FF1CF19
:10A5F000869571056105089408950E94E352A0F0C4
:10A60000BEE7B91788F4BB279F3860F41616B11D52
:10A61000672F782F8827985FF7CF8695779567956E
:10A62000B11D93959639C8F30895E894BB27662722
:10A630007727CB0197F908950E94665208F48FEFAF
:10A6400008950E9434530C94CA520E94BC5238F0B0
:10A650000E94C35220F0952311F00C948A520C945E
:10A66000B95211240C9416530E94DB5270F3959F3B
:10A67000C1F3950F50E0551F629FF001729FBB27F9
:10A68000F00DB11D639FAA27F00DB11DAA1F649F95
:10A690006627B00DA11D661F829F2227B00DA11D48
:10A6A000621F739FB00DA11D621F839FA00D611DCE
:10A6B000221F749F3327A00D611D231F849F600DEF
:10A6C000211D822F762F6A2F11249F5750409AF018
:10A6D000F1F088234AF0EE0FFF1FBB1F661F771FA4
:10A6E000881F91505040A9F79E3F510580F00C946F
:10A6F0008A520C9416535F3FE4F3983ED4F3869548
:10A7000077956795B795F795E7959F5FC1F7FE2B0E
:10A71000880F911D9695879597F90895FA01EE0F88
:10A72000FF1F309621053105A1F16115710561F416
:10A730008038BFE39B0749F168949038810561F048
:10A740008038BFEF9B0741F099234AF5FF3FE105B1
:10A750003105210519F1E8940894E795D901AA2358
:10A7600029F4AB2FBE2FF85FD0F310C0FF5F70F459
:10A77000A695E0F7F73950F019F0FF3A38F49F77D3
:10A780009F930DD00F9007FC9058089546F00C94BD
:10A79000B95260E070E080E89FE308954FE79F774B
:10A7A0005F934F933F932F930E94AD542F913F910E
:10A7B0004F915F910E9421530C940A540E94E352DE
:10A7C000E8F09E37E8F09639B8F49E3848F4672FE1
:10A7D000782F8827985FF9CF869577956795939519
:10A7E0009539D0F3B62FB1706B0F711D811D20F418
:10A7F00087957795679593950C9490520C94AB52EE
:10A800000C94165329F416F00C948A520C94155398
:10A810000C94B9520E94E352A8F39638A0F707F8B7
:10A820000F92E8942BE33AEA48EB5FE70E94375334
:10A830000F920F920F924DB75EB70F920E94F55490
:10A84000E0EAF0E00E943C544F915F91EF91FF915C
:10A85000E595EE1FFF1F49F0FE57E0684427EE0F15
:10A86000441FFA95E1F74195550B0E946F540F90E4
:10A8700007FE0C9463540895DF93CF931F930F93B7
:10A88000FF92EF92DF927B018C01689406C0DA2E72
:10A89000EF010E943453FE01E894A5912591359172
:10A8A00045915591A6F3EF010E941051FE019701C9
:10A8B000A801DA9469F7DF90EF90FF900F911F9154
:10A8C000CF91DF9108959B01AC0160E070E080E8DA
:10A8D0009FE30C946A510C948A520C94AB520E94E0
:10A8E000E352D8F39923C9F3940F511DA3F3915068
:10A8F000504094F059F0882332F0660F771F881F7C
:10A9000091505040C1F79E3F51052CF7880F911D83
:10A910009695879597F908955F3FACF0983E9CF027
:10A92000BB27869577956795B79508F4B1609395A1
:10A93000C1F7BB0F58F711F460FFE8CF6F5F7F4F8F
:10A940008F4F9F4FE3CF0C94165316F00C94AB52DD
:10A950000C94B95268940C948A520E94E352A8F362
:10A960009923C1F3AEF3DF93CF931F930F93FF921D
:10A97000C92FDD2788232AF02197660F771F881FAC
:10A98000DAF720E030E040E85FEB9FE3883920F021
:10A99000803E38F021968F770E94F950E8ECF0E085
:10A9A00004C00E94F950E5EFF0E00E943C548B0196
:10A9B000BE01EC01FB2E6F5771097595771F880B4F
:10A9C000990B0E94145228E132E741E35FE30E94B1
:10A9D0003453AF2D9801AE01FF900F911F91CF918D
:10A9E000DF910E9410510C94CA52FA01DC01AA0FA7
:10A9F000BB1F9B01AC01BF5728F4222733274427F4
:10AA0000507820C0B75190F4AB2F0024469537956D
:10AA10002795011CA395D2F3002071F0220F331F5C
:10AA2000441FB395DAF30ED00C94F85061307105E1
:10AA3000A0E88A07B94630F49B01AC016627772766
:10AA400088279078309621F0208331834283538386
:10AA50000895DB018F939F930E948350BF91AF9124
:10AA6000A29F800D911DA39F900DB29F900D112468
:10AA70000895991B79E004C0991F961708F0961B5A
:10AA8000881F7A95C9F78095089597FB072E16F4CD
:10AA9000009407D077FD09D00E94505007FC05D0E4
:10AAA0003EF4909581959F4F0895709561957F4FE5
:10AAB0000895EE0FFF1F0590F491E02D09940E9478
:10AAC000E950332312F48A1B9B0B0C9469550E94A6
:10AAD000E950B7FF0895821B930B089597FD1094DA
:10AAE000002E083098F00850232F342F452F562F72
:10AAF000672F782F892F912DF4CF159497958795EF
:10AB00007795679557954795379527950A95AAF7AD
:10AB10001124002D08950024A7FD00942A17300564
:10AB200040055005600570058005900508950F9358
:10AB30001F93CF93DF938230910510F482E090E071
:10AB4000E091092EF0910A2E30E020E0B0E0A0E084
:10AB5000309799F42115310509F44AC0281B390BA7
:10AB600024303105D8F58A819B816115710589F101
:10AB7000FB0182839383FE0111C0408151810281D8
:10AB8000138148175907E0F04817590799F41097AF
:10AB900061F012960C93129713961C933296CF0184
:10ABA000DF91CF911F910F9108950093092E10937B
:10ABB0000A2EF4CF2115310551F04217530738F012
:10ABC000A901DB019A01BD01DF01F801C1CFEF014D
:10ABD000F9CF8093092E90930A2ECDCFFE01E20F7C
:10ABE000F31F819391932250310928833983D7CF62
:10ABF0002091072E3091082E232B41F420917128AB
:10AC0000309172282093072E3093082E20916F28C0
:10AC1000309170282115310541F42DB73EB7409190
:10AC2000732850917428241B350BE091072EF09166
:10AC3000082EE217F307A0F42E1B3F0B2817390745
:10AC400078F0AC014E5F5F4F2417350748F04E0F88
:10AC50005F1F4093072E5093082E819391939FCFAF
:10AC6000F0E0E0E09CCFCF93DF930097E9F0FC01A8
:10AC7000329712821382A091092EB0910A2EED0113
:10AC800030E020E01097A1F420813181820F931FE2
:10AC90002091072E3091082E2817390709F061C03E
:10ACA000E093072EF093082EDF91CF910895EA01EB
:10ACB000CE17DF07E8F54A815B819E0141155105FA
:10ACC000B1F7E901EA83FB8349915991C40FD51F7C
:10ACD000EC17FD0761F4808191810296840F951F26
:10ACE000E90188839983828193818A839B83F0E041
:10ACF000E0E012968D919C9113970097B9F52D91F4
:10AD00003C911197CD010296820F931F2091072E3F
:10AD10003091082E2817390739F6309751F51092DF
:10AD2000092E10920A2EA093072EB093082EBCCFA6
:10AD3000C283D38340815181840F951FC817D907DF
:10AD400061F44E5F5F4F88819981480F591F40839E
:10AD500051838A819B81828393832115310509F078
:10AD6000B0CFE093092EF0930A2E9ECFFD01DC01B7
:10AD7000C0CF12821382D7CF81E090E0F8940C9478
:06AD8000C156F894FFCF5C
:10AD860001000100010001000100010001000100B5
:10AD960061F064F068F06DF071F0E9F080F083F036
:10ADA60086F089F08CF0D3EF75F077F079F07CF0CF
:10ADB6007FF082F085F088F08BF0000000008001C3
:10ADC60000000003000080030000000400001E00D5
:10ADD60000007A00000072010000E80300008813FA
:10ADE60000000000FFFF0100FFFF02000300FFFF5D
:10ADF6000400FFFF05000600070018000C0006000F
:10AE06000100FFFF0200FFFF03000400FFFF050033
:10AE1600FFFF060007000800030201000C0D0405F1
:10AE26000000000300010200000101000000000014
:10AE36000000000000000000000000000000300AD2
:10AE46002C0A00093D90D00380841E90D00324F480
:10AE5600000024F440420F00127A40420F90D003C3
:10AE6600000000000000803F0000A040A0F0A7F016
:10AE7600AFF0B6F0BFF0C7F0CEF0D6F0E0F0EBF0F2
:10AE86000504000506020401030001000102030295
:10AE96000100020304050203050400000000D205B8
:10AEA600450637052306680546055A05A11A86078D
:10AEB6007405D006000000003E0AA42A8E0A5F0A26
:10AEC6003F0A920B410BCA29980AE20BDC0B892830
:10AED600D40B00000000600D3B0D721A110D340DED
:10AEE600210D120D310EEC0DDF0DDB0DA20D830DC4
:10AEF6007B0DB10DA90DEA0CE50C201001204004D4
:10AF060010020801020102040804020104081020CC
:10AF160004082010020200050201050004010104D4
:10AF260004040303030305050303000001010000F5
:10AF360000001B174506721A711A3411D81495149D
:10AF46002C14AB13EC13C719C714B3101711C9127D
:10AF56003A13B812C4184C18ED17DF28A90F0000D1
:10AF66000000951A8D1A851A7D1A751A6F66660085
:10AF76005365742000536574207377696E672000EB
:10AF86002D002A002B00202000202030004D696370
:10AF9600726F74696D696E6773004D756C74697351
:10AFA60074657073005B005D00536574207374658F
:10AFB60070733A00537465702031207365740044D1
:10AFC60046414D205468696E670076312E3700433E
:10AFD6006F6E66696775726174696F6E005363722E
:10AFE60065656E73617665723A00436F6C6F757254
:10AFF6003A00416C6C6F7720666173743A00496E53
:10B0060076657274204C43443A005050514E3A00D3
:10B016004D4944492063683A0043616C6962726134
:10B02600746500506C6179204332004F4B20280034
:10B036002900506C6179204334004F4B00446F6EF9
:10B0460065004661696C65640053657420737465B8
:10B0560070733A200042504D3A20004F6E004F6602
:10B066006600426C75650052656400416C6C003880
:10B0760000390031300031310031320031330031D6
:10B086003400313500313600496E742E004578742F
:10B096002E004D494449003234004E6F726D616C8A
:10B0A600005265766572736500426F756E63650062
:10B0B6004F64642F4576656E0053687566666C65E9
:10B0C6000052616E646F6D004356204D6F646500DB
:10B0D6004D494449204D6F6465005365742073746F
:0BB0E60065702031005377696E670031
:10B0F1001027FFFFFFFF3C028B01189DF07FF08CB2
:10B10100F00024F400015A00010200FFFF0000805A
:10B111003F010001000100010001000100010001E7
:10B12100000000803FFFFF010000484300000800CD
:10B131000000010000000078000000000000010094
:10B1410002000300040005000600070000000000E3
:10B15100000000FFFFFFFF010000000100000000F0
:06B16100000B2E8000002F
:00000001FF
